################################################################################
#                                                                              #
#      IAR Universal Linker V6.1.3.56                                          #
#                                                                              #
#           Link time     =  10/Feb/2016  17:35:54                             #
#           Target CPU    =  MSP430                                            #
#           List file     =  C:\Users\a0415888\Documents\pwd\GIT_REPOS\TDC7200 #
#                            \tdc7200evm_fw\Debug\List\demo2_tdc720x_usb.map   #
#           Output file 1 =  C:\Users\a0415888\Documents\pwd\GIT_REPOS\TDC7200 #
#                            \tdc7200evm_fw\Debug\Exe\demo2_tdc720x_usb.d43    #
#                            Format: debug                                     #
#                            UBROF version 10.0.6                              #
#                            Using library modules for C-SPY (-rt)             #
#           Output file 2 =  C:\Users\a0415888\Documents\pwd\GIT_REPOS\TDC7200 #
#                            \tdc7200evm_fw\Debug\Exe\demo2_tdc720x_usb.txt    #
#                            Format: msp430_txt                                #
#           Command line  =  C:\Users\a0415888\Documents\pwd\GIT_REPOS\TDC7200 #
#                            \tdc7200evm_fw\Debug\Obj\adc10_a.r43              #
#                            C:\Users\a0415888\Documents\pwd\GIT_REPOS\TDC7200 #
#                            \tdc7200evm_fw\Debug\Obj\adc12_a.r43              #
#                            C:\Users\a0415888\Documents\pwd\GIT_REPOS\TDC7200 #
#                            \tdc7200evm_fw\Debug\Obj\aes.r43                  #
#                            C:\Users\a0415888\Documents\pwd\GIT_REPOS\TDC7200 #
#                            \tdc7200evm_fw\Debug\Obj\battbak.r43              #
#                            C:\Users\a0415888\Documents\pwd\GIT_REPOS\TDC7200 #
#                            \tdc7200evm_fw\Debug\Obj\comp_b.r43               #
#                            C:\Users\a0415888\Documents\pwd\GIT_REPOS\TDC7200 #
#                            \tdc7200evm_fw\Debug\Obj\crc.r43                  #
#                            C:\Users\a0415888\Documents\pwd\GIT_REPOS\TDC7200 #
#                            \tdc7200evm_fw\Debug\Obj\dac12_a.r43              #
#                            C:\Users\a0415888\Documents\pwd\GIT_REPOS\TDC7200 #
#                            \tdc7200evm_fw\Debug\Obj\descriptors.r43          #
#                            C:\Users\a0415888\Documents\pwd\GIT_REPOS\TDC7200 #
#                            \tdc7200evm_fw\Debug\Obj\dma.r43                  #
#                            C:\Users\a0415888\Documents\pwd\GIT_REPOS\TDC7200 #
#                            \tdc7200evm_fw\Debug\Obj\eusci_a_spi.r43          #
#                            C:\Users\a0415888\Documents\pwd\GIT_REPOS\TDC7200 #
#                            \tdc7200evm_fw\Debug\Obj\eusci_a_uart.r43         #
#                            C:\Users\a0415888\Documents\pwd\GIT_REPOS\TDC7200 #
#                            \tdc7200evm_fw\Debug\Obj\eusci_b_i2c.r43          #
#                            C:\Users\a0415888\Documents\pwd\GIT_REPOS\TDC7200 #
#                            \tdc7200evm_fw\Debug\Obj\eusci_b_spi.r43          #
#                            C:\Users\a0415888\Documents\pwd\GIT_REPOS\TDC7200 #
#                            \tdc7200evm_fw\Debug\Obj\flashctl.r43             #
#                            C:\Users\a0415888\Documents\pwd\GIT_REPOS\TDC7200 #
#                            \tdc7200evm_fw\Debug\Obj\gpio.r43                 #
#                            C:\Users\a0415888\Documents\pwd\GIT_REPOS\TDC7200 #
#                            \tdc7200evm_fw\Debug\Obj\HAL_FLASH.r43            #
#                            C:\Users\a0415888\Documents\pwd\GIT_REPOS\TDC7200 #
#                            \tdc7200evm_fw\Debug\Obj\HAL_PMAP.r43             #
#                            C:\Users\a0415888\Documents\pwd\GIT_REPOS\TDC7200 #
#                            \tdc7200evm_fw\Debug\Obj\HAL_PMM.r43              #
#                            C:\Users\a0415888\Documents\pwd\GIT_REPOS\TDC7200 #
#                            \tdc7200evm_fw\Debug\Obj\HAL_TLV.r43              #
#                            C:\Users\a0415888\Documents\pwd\GIT_REPOS\TDC7200 #
#                            \tdc7200evm_fw\Debug\Obj\HAL_UCS.r43              #
#                            C:\Users\a0415888\Documents\pwd\GIT_REPOS\TDC7200 #
#                            \tdc7200evm_fw\Debug\Obj\host_interface.r43       #
#                            C:\Users\a0415888\Documents\pwd\GIT_REPOS\TDC7200 #
#                            \tdc7200evm_fw\Debug\Obj\ldopwr.r43               #
#                            C:\Users\a0415888\Documents\pwd\GIT_REPOS\TDC7200 #
#                            \tdc7200evm_fw\Debug\Obj\main.r43                 #
#                            C:\Users\a0415888\Documents\pwd\GIT_REPOS\TDC7200 #
#                            \tdc7200evm_fw\Debug\Obj\mpy32.r43                #
#                            C:\Users\a0415888\Documents\pwd\GIT_REPOS\TDC7200 #
#                            \tdc7200evm_fw\Debug\Obj\pmap.r43                 #
#                            C:\Users\a0415888\Documents\pwd\GIT_REPOS\TDC7200 #
#                            \tdc7200evm_fw\Debug\Obj\pmm.r43                  #
#                            C:\Users\a0415888\Documents\pwd\GIT_REPOS\TDC7200 #
#                            \tdc7200evm_fw\Debug\Obj\ram.r43                  #
#                            C:\Users\a0415888\Documents\pwd\GIT_REPOS\TDC7200 #
#                            \tdc7200evm_fw\Debug\Obj\ref.r43                  #
#                            C:\Users\a0415888\Documents\pwd\GIT_REPOS\TDC7200 #
#                            \tdc7200evm_fw\Debug\Obj\rtc_a.r43                #
#                            C:\Users\a0415888\Documents\pwd\GIT_REPOS\TDC7200 #
#                            \tdc7200evm_fw\Debug\Obj\rtc_b.r43                #
#                            C:\Users\a0415888\Documents\pwd\GIT_REPOS\TDC7200 #
#                            \tdc7200evm_fw\Debug\Obj\rtc_c.r43                #
#                            C:\Users\a0415888\Documents\pwd\GIT_REPOS\TDC7200 #
#                            \tdc7200evm_fw\Debug\Obj\sd24_b.r43               #
#                            C:\Users\a0415888\Documents\pwd\GIT_REPOS\TDC7200 #
#                            \tdc7200evm_fw\Debug\Obj\sfr.r43                  #
#                            C:\Users\a0415888\Documents\pwd\GIT_REPOS\TDC7200 #
#                            \tdc7200evm_fw\Debug\Obj\sysctl.r43               #
#                            C:\Users\a0415888\Documents\pwd\GIT_REPOS\TDC7200 #
#                            \tdc7200evm_fw\Debug\Obj\tdc720x_calculation.r43  #
#                            C:\Users\a0415888\Documents\pwd\GIT_REPOS\TDC7200 #
#                            \tdc7200evm_fw\Debug\Obj\tdc720x_measurement_cont #
#                            rol.r43                                           #
#                            C:\Users\a0415888\Documents\pwd\GIT_REPOS\TDC7200 #
#                            \tdc7200evm_fw\Debug\Obj\tdc720x_mode1_lt12ns.r43 #
#                            C:\Users\a0415888\Documents\pwd\GIT_REPOS\TDC7200 #
#                            \tdc7200evm_fw\Debug\Obj\tec.r43                  #
#                            C:\Users\a0415888\Documents\pwd\GIT_REPOS\TDC7200 #
#                            \tdc7200evm_fw\Debug\Obj\TI_MSP430_spi_USCIB0_5xx #
#                            .r43                                              #
#                            C:\Users\a0415888\Documents\pwd\GIT_REPOS\TDC7200 #
#                            \tdc7200evm_fw\Debug\Obj\timer_a.r43              #
#                            C:\Users\a0415888\Documents\pwd\GIT_REPOS\TDC7200 #
#                            \tdc7200evm_fw\Debug\Obj\timer_b.r43              #
#                            C:\Users\a0415888\Documents\pwd\GIT_REPOS\TDC7200 #
#                            \tdc7200evm_fw\Debug\Obj\timer_d.r43              #
#                            C:\Users\a0415888\Documents\pwd\GIT_REPOS\TDC7200 #
#                            \tdc7200evm_fw\Debug\Obj\timer_queue.r43          #
#                            C:\Users\a0415888\Documents\pwd\GIT_REPOS\TDC7200 #
#                            \tdc7200evm_fw\Debug\Obj\tlv.r43                  #
#                            C:\Users\a0415888\Documents\pwd\GIT_REPOS\TDC7200 #
#                            \tdc7200evm_fw\Debug\Obj\uart_commn.r43           #
#                            C:\Users\a0415888\Documents\pwd\GIT_REPOS\TDC7200 #
#                            \tdc7200evm_fw\Debug\Obj\ucs.r43                  #
#                            C:\Users\a0415888\Documents\pwd\GIT_REPOS\TDC7200 #
#                            \tdc7200evm_fw\Debug\Obj\usb.r43                  #
#                            C:\Users\a0415888\Documents\pwd\GIT_REPOS\TDC7200 #
#                            \tdc7200evm_fw\Debug\Obj\UsbCdc.r43               #
#                            C:\Users\a0415888\Documents\pwd\GIT_REPOS\TDC7200 #
#                            \tdc7200evm_fw\Debug\Obj\usbConstructs.r43        #
#                            C:\Users\a0415888\Documents\pwd\GIT_REPOS\TDC7200 #
#                            \tdc7200evm_fw\Debug\Obj\usbdma.r43               #
#                            C:\Users\a0415888\Documents\pwd\GIT_REPOS\TDC7200 #
#                            \tdc7200evm_fw\Debug\Obj\usbEventHandling.r43     #
#                            C:\Users\a0415888\Documents\pwd\GIT_REPOS\TDC7200 #
#                            \tdc7200evm_fw\Debug\Obj\UsbIsr.r43               #
#                            C:\Users\a0415888\Documents\pwd\GIT_REPOS\TDC7200 #
#                            \tdc7200evm_fw\Debug\Obj\usci_a_spi.r43           #
#                            C:\Users\a0415888\Documents\pwd\GIT_REPOS\TDC7200 #
#                            \tdc7200evm_fw\Debug\Obj\usci_a_uart.r43          #
#                            C:\Users\a0415888\Documents\pwd\GIT_REPOS\TDC7200 #
#                            \tdc7200evm_fw\Debug\Obj\usci_b_i2c.r43           #
#                            C:\Users\a0415888\Documents\pwd\GIT_REPOS\TDC7200 #
#                            \tdc7200evm_fw\Debug\Obj\usci_b_spi.r43           #
#                            C:\Users\a0415888\Documents\pwd\GIT_REPOS\TDC7200 #
#                            \tdc7200evm_fw\Debug\Obj\wdt_a.r43                #
#                            -o                                                #
#                            C:\Users\a0415888\Documents\pwd\GIT_REPOS\TDC7200 #
#                            \tdc7200evm_fw\Debug\Exe\demo2_tdc720x_usb.d43    #
#                            -l                                                #
#                            C:\Users\a0415888\Documents\pwd\GIT_REPOS\TDC7200 #
#                            \tdc7200evm_fw\Debug\List\demo2_tdc720x_usb.map   #
#                            -xmsn                                             #
#                            "-IC:\Program Files (x86)\IAR Systems\Embedded Wo #
#                            rkbench 7.0\430\LIB\"                             #
#                            -f                                                #
#                            "C:\Program Files (x86)\IAR Systems\Embedded Work #
#                            bench 7.0\430\config\linker\lnk430f5529.xcl"      #
#                            (-cmsp430 -D?CPU30_OFFSET=2 -QCODE_I=CODE_ID      #
#                            -QTLS16_I=TLS16_ID -D__iar_HWMUL=4C0              #
#                            -Z(CONST)INFO=1800-19FF                           #
#                            -Z(CONST)INFOA=1980-19FF                          #
#                            -Z(CONST)INFOB=1900-197F                          #
#                            -Z(CONST)INFOC=1880-18FF                          #
#                            -Z(CONST)INFOD=1800-187F                          #
#                            -Z(DATA)DATA16_I,DATA16_Z,DATA16_N,TLS16_I=2400-4 #
#                            3FF                                               #
#                            -Z(DATA)DATA16_HEAP+_DATA16_HEAP_SIZE             #
#                            -Z(DATA)CODE_I                                    #
#                            -Z(DATA)DATA20_I,DATA20_Z,DATA20_N,DATA20_HEAP+_D #
#                            ATA20_HEAP_SIZE                                   #
#                            -Z(DATA)CSTACK+_STACK_SIZE#                       #
#                            -Z(CONST)DATA16_C,DATA16_ID,TLS16_ID,DIFUNCT,CHEC #
#                            KSUM=4400-FF7F                                    #
#                            -Z(CODE)CSTART,ISR_CODE,CODE16=4400-FF7F          #
#                            -P(CODE)CODE=4400-FF7F,10000-243FF                #
#                            -Z(CONST)DATA20_C,DATA20_ID,CODE_ID=4400-FF7F,100 #
#                            40-243FF                                          #
#                            -Z(CODE)INTVEC=FF80-FFFF                          #
#                            -Z(CODE)RESET=FFFE-FFFF) -f                       #
#                            "C:\Program Files (x86)\IAR Systems\Embedded Work #
#                            bench 7.0\430\config\linker\multiplier32.xcl"     #
#                            (-e?Mul8Hw=?Mul8 -e?Mul16Hw=?Mul16                #
#                            -e?Mul16to32uHw=?Mul16to32u                       #
#                            -e?Mul16to32sHw=?Mul16to32s -e?Mul32Hw32=?Mul32   #
#                            -e?Mul64Hw32=_Mul64i                              #
#                            -e?Mul32u32uto64iHw32=_Mul32u32uto64i             #
#                            -e?Mul32fHw=_Mul32f -e_Mul64fHwPtr=_Mul64fPtr)    #
#                            -D_STACK_SIZE=A0 -rt                              #
#                            "C:\Program Files (x86)\IAR Systems\Embedded Work #
#                            bench 7.0\430\lib\dlib\dl430xlsfn.r43"            #
#                            -D_DATA16_HEAP_SIZE=A0                            #
#                            -Omsp430_txt=C:\Users\a0415888\Documents\pwd\GIT_ #
#                            REPOS\TDC7200\tdc7200evm_fw\Debug\Exe\demo2_tdc72 #
#                            0x_usb.txt                                        #
#                            -s __program_start -D_DATA20_HEAP_SIZE=50         #
#                                                                              #
#                           Copyright (C) 1987-2014 IAR Systems AB.            #
################################################################################





                ****************************************
                *                                      *
                *           CROSS REFERENCE            *
                *                                      *
                ****************************************

       Program entry at :           4690  Relocatable, from module : ?cstart




                ****************************************
                *                                      *
                *            RUNTIME MODEL             *
                *                                      *
                ****************************************

  __Heap_Handler             = Basic
  __SystemLibrary            = DLib
  __code_model               = large
  __core                     = 430X
  __data_model               = small
  __dlib_file_descriptor     = 0
  __dlib_full_locale_support = 0
  __double_size              = 32
  __pic                      = no
  __reg_r4                   = free
  __reg_r5                   = free
  __rt_version               = 3

                ****************************************
                *                                      *
                *    AUTOMATIC SYMBOL REDIRECTIONS     *
                *                                      *
                ****************************************

       All references to: _Printf
         were redirected to: _PrintfLargeNoMb



                ****************************************
                *                                      *
                *              MODULE MAP              *
                *                                      *
                ****************************************


  DEFINED ABSOLUTE ENTRIES
    *************************************************************************

  DEFINED ABSOLUTE ENTRIES
  PROGRAM MODULE, NAME : ?ABS_ENTRY_MOD

Absolute parts
           ENTRY                   ADDRESS         REF BY
           =====                   =======         ======
           _DATA20_HEAP_SIZE       0050 
           _DATA16_HEAP_SIZE       00A0 
           _STACK_SIZE             00A0 
           __iar_HWMUL             04C0            ?Mul32Hw32 (?Mul32Hw32)
                                                   ?Mul32fHw (?Mul32fHw)
                                                   USB_determineFreq (usb)
           ?CPU30_OFFSET           0002 
    *************************************************************************

  FILE NAME : C:\Users\a0415888\Documents\pwd\GIT_REPOS\TDC7200\tdc7200evm_fw\Debug\Obj\adc10_a.r43
    *************************************************************************

  FILE NAME : C:\Users\a0415888\Documents\pwd\GIT_REPOS\TDC7200\tdc7200evm_fw\Debug\Obj\adc12_a.r43
    *************************************************************************

  FILE NAME : C:\Users\a0415888\Documents\pwd\GIT_REPOS\TDC7200\tdc7200evm_fw\Debug\Obj\aes.r43
    *************************************************************************

  FILE NAME : C:\Users\a0415888\Documents\pwd\GIT_REPOS\TDC7200\tdc7200evm_fw\Debug\Obj\battbak.r43
    *************************************************************************

  FILE NAME : C:\Users\a0415888\Documents\pwd\GIT_REPOS\TDC7200\tdc7200evm_fw\Debug\Obj\comp_b.r43
    *************************************************************************

  FILE NAME : C:\Users\a0415888\Documents\pwd\GIT_REPOS\TDC7200\tdc7200evm_fw\Debug\Obj\crc.r43
    *************************************************************************

  FILE NAME : C:\Users\a0415888\Documents\pwd\GIT_REPOS\TDC7200\tdc7200evm_fw\Debug\Obj\dac12_a.r43
    *************************************************************************

  FILE NAME : C:\Users\a0415888\Documents\pwd\GIT_REPOS\TDC7200\tdc7200evm_fw\Debug\Obj\descriptors.r43
  PROGRAM MODULE, NAME : descriptors

  SEGMENTS IN THE MODULE
  ======================
DATA16_C
  Relative segment, address: 4536 - 4547 (0x12 bytes), align: 0
  Segment part 2.
           ENTRY                   ADDRESS         REF BY
           =====                   =======         ======
           abromDeviceDescriptor   4536            usbGetDeviceDescriptor (usb)
    -------------------------------------------------------------------------
DATA16_C
  Relative segment, address: 4548 - 458A (0x43 bytes), align: 0
  Segment part 3.
           ENTRY                   ADDRESS         REF BY
           =====                   =======         ======
           abromConfigurationDescriptorGroup
                                   4548            usbGetConfigurationDescriptor (usb)
                                                   usbGetDeviceStatus (usb)
    -------------------------------------------------------------------------
DATA16_C
  Relative segment, address: 458B - 4618 (0x8e bytes), align: 0
  Segment part 4.
           ENTRY                   ADDRESS         REF BY
           =====                   =======         ======
           abromStringDescriptor   458B            usbGetStringDescriptor (usb)
    -------------------------------------------------------------------------
DATA16_C
  Relative segment, address: 4400 - 440F (0x10 bytes), align: 1
  Segment part 5.
           ENTRY                   ADDRESS         REF BY
           =====                   =======         ======
           stUsbHandle             4400            CdcToBufferFromHost (UsbCdc)
                                                   CdcToHostFromBuffer (UsbCdc)
                                                   USBCDC_abortSend (UsbCdc)
                                                   USBCDC_getBytesInUSBBuffer (UsbCdc)
                                                   USBCDC_getInterfaceStatus (UsbCdc)
                                                   USBCDC_receiveData (UsbCdc)
                                                   USBCDC_sendData (UsbCdc)
                                                   USB_reset (usb)
    -------------------------------------------------------------------------
DATA16_C
  Relative segment, address: 4410 - 4519 (0x10a bytes), align: 1
  Segment part 6.
           ENTRY                   ADDRESS         REF BY
           =====                   =======         ======
           tUsbRequestList         4410            usbDecodeAndProcessUsbRequest (usb)

    *************************************************************************

  FILE NAME : C:\Users\a0415888\Documents\pwd\GIT_REPOS\TDC7200\tdc7200evm_fw\Debug\Obj\dma.r43
  PROGRAM MODULE, NAME : dma

  SEGMENTS IN THE MODULE
  ======================
<CODE> 1 (was CODE)
  Relative segment, address: 7BB6 - 7C3D (0x88 bytes), align: 1
  Segment part 21.
           ENTRY                   ADDRESS         REF BY
           =====                   =======         ======
           DMA_init                7BB6            USB_initMemcpy (usbdma)
               CSTACK = 00000000 ( 00000004 )
    -------------------------------------------------------------------------
<CODE> 1 (was CODE)
  Relative segment, address: 9280 - 928B (0xc bytes), align: 1
  Segment part 20.
           ENTRY                   ADDRESS         REF BY
           =====                   =======         ======
           DMA_setTransferSize     9280            memcpyDMA (usbdma)
               CSTACK = 00000000 ( 00000004 )
    -------------------------------------------------------------------------
<CODE> 1 (was CODE)
  Relative segment, address: 8DA4 - 8DCD (0x2a bytes), align: 1
  Segment part 18.
           ENTRY                   ADDRESS         REF BY
           =====                   =======         ======
           DMA_setSrcAddress       8DA4            memcpyDMA (usbdma)
               CSTACK = 00000000 ( 00000006 )
    -------------------------------------------------------------------------
<CODE> 1 (was CODE)
  Relative segment, address: 8CCC - 8CF7 (0x2c bytes), align: 1
  Segment part 17.
           ENTRY                   ADDRESS         REF BY
           =====                   =======         ======
           DMA_setDstAddress       8CCC            memcpyDMA (usbdma)
               CSTACK = 00000000 ( 00000006 )
    -------------------------------------------------------------------------
<CODE> 1 (was CODE)
  Relative segment, address: 922A - 9237 (0xe bytes), align: 1
  Segment part 16.
           ENTRY                   ADDRESS         REF BY
           =====                   =======         ======
           DMA_enableTransfers     922A            memcpyDMA (usbdma)
               CSTACK = 00000000 ( 00000004 )
    -------------------------------------------------------------------------
<CODE> 1 (was CODE)
  Relative segment, address: 91F2 - 91FF (0xe bytes), align: 1
  Segment part 15.
           ENTRY                   ADDRESS         REF BY
           =====                   =======         ======
           DMA_disableTransfers    91F2            memcpyDMA (usbdma)
               CSTACK = 00000000 ( 00000004 )
    -------------------------------------------------------------------------
<CODE> 1 (was CODE)
  Relative segment, address: 9268 - 9273 (0xc bytes), align: 1
  Segment part 14.
           ENTRY                   ADDRESS         REF BY
           =====                   =======         ======
           DMA_startTransfer       9268            memcpyDMA (usbdma)
               CSTACK = 00000000 ( 00000004 )
    -------------------------------------------------------------------------
<CODE> 1 (was CODE)
  Relative segment, address: 9250 - 925B (0xc bytes), align: 1
  Segment part 11.
           ENTRY                   ADDRESS         REF BY
           =====                   =======         ======
           DMA_getInterruptStatus
                                   9250            memcpyDMA (usbdma)
               CSTACK = 00000000 ( 00000004 )
    -------------------------------------------------------------------------
<CODE> 1 (was CODE)
  Relative segment, address: 92E6 - 92EB (0x6 bytes), align: 1
  Segment part 7.
           ENTRY                   ADDRESS         REF BY
           =====                   =======         ======
           DMA_disableTransferDuringReadModifyWrite
                                   92E6            memcpyDMA (usbdma)
               CSTACK = 00000000 ( 00000004 )
    -------------------------------------------------------------------------
<CODE> 1 (was CODE)
  Relative segment, address: 92EC - 92F1 (0x6 bytes), align: 1
  Segment part 6.
           ENTRY                   ADDRESS         REF BY
           =====                   =======         ======
           DMA_enableTransferDuringReadModifyWrite
                                   92EC            memcpyDMA (usbdma)
               CSTACK = 00000000 ( 00000004 )

    *************************************************************************

  FILE NAME : C:\Users\a0415888\Documents\pwd\GIT_REPOS\TDC7200\tdc7200evm_fw\Debug\Obj\eusci_a_spi.r43
    *************************************************************************

  FILE NAME : C:\Users\a0415888\Documents\pwd\GIT_REPOS\TDC7200\tdc7200evm_fw\Debug\Obj\eusci_a_uart.r43
    *************************************************************************

  FILE NAME : C:\Users\a0415888\Documents\pwd\GIT_REPOS\TDC7200\tdc7200evm_fw\Debug\Obj\eusci_b_i2c.r43
    *************************************************************************

  FILE NAME : C:\Users\a0415888\Documents\pwd\GIT_REPOS\TDC7200\tdc7200evm_fw\Debug\Obj\eusci_b_spi.r43
    *************************************************************************

  FILE NAME : C:\Users\a0415888\Documents\pwd\GIT_REPOS\TDC7200\tdc7200evm_fw\Debug\Obj\flashctl.r43
    *************************************************************************

  FILE NAME : C:\Users\a0415888\Documents\pwd\GIT_REPOS\TDC7200\tdc7200evm_fw\Debug\Obj\gpio.r43
  PROGRAM MODULE, NAME : gpio

  SEGMENTS IN THE MODULE
  ======================
DATA16_C
  Relative segment, address: 451A - 4535 (0x1c bytes), align: 1
  Segment part 2.             Intra module refs:   GPIO_setAsPeripheralModuleFunctionOutputPin
           LOCAL                   ADDRESS         
           =====                   =======         
           GPIO_PORT_TO_BASE       451A 
    -------------------------------------------------------------------------
<CODE> 1 (was CODE)
  Relative segment, address: 8D7A - 8DA3 (0x2a bytes), align: 1
  Segment part 16.
           ENTRY                   ADDRESS         REF BY
           =====                   =======         ======
           GPIO_setAsPeripheralModuleFunctionOutputPin
                                   8D7A            USB_enable (usb)
               CSTACK = 00000000 ( 00000004 )

    *************************************************************************

  FILE NAME : C:\Users\a0415888\Documents\pwd\GIT_REPOS\TDC7200\tdc7200evm_fw\Debug\Obj\HAL_FLASH.r43
  PROGRAM MODULE, NAME : HAL_FLASH

  SEGMENTS IN THE MODULE
  ======================
DATA16_AN
  Relative segment, address: 0140 - 0141 (0x2 bytes), align: 0
  Segment part 1. ROOT 
           ENTRY                   ADDRESS         REF BY
           =====                   =======         ======
           _A_FCTL1_L              0140 
           LOCAL                   ADDRESS         
           =====                   =======         
           FCTL1                   0140 
           FCTL1_H                 0141 
           FCTL1_L                 0140 
    -------------------------------------------------------------------------
DATA16_AN
  Relative segment, address: 0144 - 0145 (0x2 bytes), align: 0
  Segment part 2. ROOT 
           ENTRY                   ADDRESS         REF BY
           =====                   =======         ======
           _A_FCTL3_L              0144 
           LOCAL                   ADDRESS         
           =====                   =======         
           FCTL3                   0144 
           FCTL3_H                 0145 
           FCTL3_L                 0144 

    *************************************************************************

  FILE NAME : C:\Users\a0415888\Documents\pwd\GIT_REPOS\TDC7200\tdc7200evm_fw\Debug\Obj\HAL_PMAP.r43
  PROGRAM MODULE, NAME : HAL_PMAP

  SEGMENTS IN THE MODULE
  ======================
DATA16_AN
  Relative segment, address: 01C0 - 01C1 (0x2 bytes), align: 0
  Segment part 1. ROOT 
           ENTRY                   ADDRESS         REF BY
           =====                   =======         ======
           _A_PMAPKEYID_L          01C0 
           LOCAL                   ADDRESS         
           =====                   =======         
           PMAPKEYID               01C0 
           PMAPKEYID_H             01C1 
           PMAPKEYID_L             01C0 
    -------------------------------------------------------------------------
DATA16_AN
  Relative segment, address: 01C2 - 01C3 (0x2 bytes), align: 0
  Segment part 2. ROOT 
           ENTRY                   ADDRESS         REF BY
           =====                   =======         ======
           _A_PMAPCTL_L            01C2 
           LOCAL                   ADDRESS         
           =====                   =======         
           PMAPCTL                 01C2 
           PMAPCTL_H               01C3 
           PMAPCTL_L               01C2 

    *************************************************************************

  FILE NAME : C:\Users\a0415888\Documents\pwd\GIT_REPOS\TDC7200\tdc7200evm_fw\Debug\Obj\HAL_PMM.r43
  PROGRAM MODULE, NAME : HAL_PMM

  SEGMENTS IN THE MODULE
  ======================
DATA16_AN
  Relative segment, address: 0120 - 0121 (0x2 bytes), align: 0
  Segment part 1. ROOT        Intra module refs:   SetVCore
                                                   SetVCoreDown
                                                   SetVCoreUp
           ENTRY                   ADDRESS         REF BY
           =====                   =======         ======
           _A_PMMCTL0_L            0120 
           LOCAL                   ADDRESS         
           =====                   =======         
           PMMCTL0                 0120 
           PMMCTL0_H               0121 
           PMMCTL0_L               0120 
    -------------------------------------------------------------------------
DATA16_AN
  Relative segment, address: 0124 - 0125 (0x2 bytes), align: 0
  Segment part 2. ROOT        Intra module refs:   SetVCoreDown
                                                   SetVCoreUp
           ENTRY                   ADDRESS         REF BY
           =====                   =======         ======
           _A_SVSMHCTL_L           0124 
           LOCAL                   ADDRESS         
           =====                   =======         
           SVSMHCTL                0124 
           SVSMHCTL_H              0125 
           SVSMHCTL_L              0124 
    -------------------------------------------------------------------------
DATA16_AN
  Relative segment, address: 0126 - 0127 (0x2 bytes), align: 0
  Segment part 3. ROOT        Intra module refs:   SetVCoreDown
                                                   SetVCoreUp
           ENTRY                   ADDRESS         REF BY
           =====                   =======         ======
           _A_SVSMLCTL_L           0126 
           LOCAL                   ADDRESS         
           =====                   =======         
           SVSMLCTL                0126 
           SVSMLCTL_H              0127 
           SVSMLCTL_L              0126 
    -------------------------------------------------------------------------
DATA16_AN
  Relative segment, address: 012C - 012D (0x2 bytes), align: 0
  Segment part 4. ROOT        Intra module refs:   SetVCoreDown
                                                   SetVCoreUp
           ENTRY                   ADDRESS         REF BY
           =====                   =======         ======
           _A_PMMIFG_L             012C 
           LOCAL                   ADDRESS         
           =====                   =======         
           PMMIFG                  012C 
           PMMIFG_H                012D 
           PMMIFG_L                012C 
    -------------------------------------------------------------------------
DATA16_AN
  Relative segment, address: 012E - 012F (0x2 bytes), align: 0
  Segment part 5. ROOT        Intra module refs:   SetVCoreDown
                                                   SetVCoreUp
           ENTRY                   ADDRESS         REF BY
           =====                   =======         ======
           _A_PMMRIE_L             012E 
           LOCAL                   ADDRESS         
           =====                   =======         
           PMMRIE                  012E 
           PMMRIE_H                012F 
           PMMRIE_L                012E 
    -------------------------------------------------------------------------
<CODE> 1 (was CODE)
  Relative segment, address: 6DEE - 6EC9 (0xdc bytes), align: 1
  Segment part 9.             Intra module refs:   SetVCore
           LOCAL                   ADDRESS         
           =====                   =======         
           SetVCoreUp              6DEE 
               CSTACK = 00000000 ( 00000008 )
    -------------------------------------------------------------------------
<CODE> 1 (was CODE)
  Relative segment, address: 7436 - 74D3 (0x9e bytes), align: 1
  Segment part 8.             Intra module refs:   SetVCore
           LOCAL                   ADDRESS         
           =====                   =======         
           SetVCoreDown            7436 
               CSTACK = 00000000 ( 0000000C )
    -------------------------------------------------------------------------
<CODE> 1 (was CODE)
  Relative segment, address: 86E0 - 872B (0x4c bytes), align: 1
  Segment part 7.
           ENTRY                   ADDRESS         REF BY
           =====                   =======         ======
           SetVCore                86E0            InitMCU (main)
               calls direct
               CSTACK = 00000000 ( 00000008 )

    *************************************************************************

  FILE NAME : C:\Users\a0415888\Documents\pwd\GIT_REPOS\TDC7200\tdc7200evm_fw\Debug\Obj\HAL_TLV.r43
    *************************************************************************

  FILE NAME : C:\Users\a0415888\Documents\pwd\GIT_REPOS\TDC7200\tdc7200evm_fw\Debug\Obj\HAL_UCS.r43
  PROGRAM MODULE, NAME : HAL_UCS

  SEGMENTS IN THE MODULE
  ======================
DATA16_AN
  Relative segment, address: 0102 - 0103 (0x2 bytes), align: 0
  Segment part 1. ROOT        Intra module refs:   Init_Clock (main)
                                                   UNMI_ISR (main)
           ENTRY                   ADDRESS         REF BY
           =====                   =======         ======
           _A_SFRIFG1_L            0102 
           LOCAL                   ADDRESS         
           =====                   =======         
           SFRIFG1                 0102 
           SFRIFG1_H               0103 
           SFRIFG1_L               0102 
    -------------------------------------------------------------------------
DATA16_AN
  Relative segment, address: 0160 - 0161 (0x2 bytes), align: 0
  Segment part 2. ROOT        Intra module refs:   Init_Clock (main)
           ENTRY                   ADDRESS         REF BY
           =====                   =======         ======
           _A_UCSCTL0_L            0160 
           LOCAL                   ADDRESS         
           =====                   =======         
           UCSCTL0                 0160 
           UCSCTL0_H               0161 
           UCSCTL0_L               0160 
    -------------------------------------------------------------------------
DATA16_AN
  Relative segment, address: 0162 - 0163 (0x2 bytes), align: 0
  Segment part 3. ROOT        Intra module refs:   Init_Clock (main)
           ENTRY                   ADDRESS         REF BY
           =====                   =======         ======
           _A_UCSCTL1_L            0162 
           LOCAL                   ADDRESS         
           =====                   =======         
           UCSCTL1                 0162 
           UCSCTL1_H               0163 
           UCSCTL1_L               0162 
    -------------------------------------------------------------------------
DATA16_AN
  Relative segment, address: 0164 - 0165 (0x2 bytes), align: 0
  Segment part 4. ROOT        Intra module refs:   Init_Clock (main)
                                                   USB_determineFreq (usb)
           ENTRY                   ADDRESS         REF BY
           =====                   =======         ======
           _A_UCSCTL2_L            0164 
           LOCAL                   ADDRESS         
           =====                   =======         
           UCSCTL2                 0164 
           UCSCTL2_H               0165 
           UCSCTL2_L               0164 
    -------------------------------------------------------------------------
DATA16_AN
  Relative segment, address: 0168 - 0169 (0x2 bytes), align: 0
  Segment part 5. ROOT        Intra module refs:   Init_Clock (main)
                                                   USB_determineFreq (usb)
           ENTRY                   ADDRESS         REF BY
           =====                   =======         ======
           _A_UCSCTL4_L            0168 
           LOCAL                   ADDRESS         
           =====                   =======         
           UCSCTL4                 0168 
           UCSCTL4_H               0169 
           UCSCTL4_L               0168 
    -------------------------------------------------------------------------
DATA16_AN
  Relative segment, address: 016C - 016D (0x2 bytes), align: 0
  Segment part 6. ROOT        Intra module refs:   Init_Clock (main)
           ENTRY                   ADDRESS         REF BY
           =====                   =======         ======
           _A_UCSCTL6_L            016C 
           LOCAL                   ADDRESS         
           =====                   =======         
           UCSCTL6                 016C 
           UCSCTL6_H               016D 
           UCSCTL6_L               016C 
    -------------------------------------------------------------------------
DATA16_AN
  Relative segment, address: 016E - 016F (0x2 bytes), align: 0
  Segment part 7. ROOT        Intra module refs:   Init_Clock (main)
                                                   UNMI_ISR (main)
           ENTRY                   ADDRESS         REF BY
           =====                   =======         ======
           _A_UCSCTL7_L            016E 
           LOCAL                   ADDRESS         
           =====                   =======         
           UCSCTL7                 016E 
           UCSCTL7_H               016F 
           UCSCTL7_L               016E 

    *************************************************************************

  FILE NAME : C:\Users\a0415888\Documents\pwd\GIT_REPOS\TDC7200\tdc7200evm_fw\Debug\Obj\host_interface.r43
  PROGRAM MODULE, NAME : host_interface

  SEGMENTS IN THE MODULE
  ======================
DATA16_AN
  Relative segment, address: 0202 - 0203 (0x2 bytes), align: 0
  Segment part 1. ROOT        Intra module refs:   Init_Clock (main)
                                                   TI_TDC720x_SPIAllReadReg (TI_MSP430_spi_USCIB0_5xx)
                                                   TI_TDC720x_SPIAllReadReg_BothTDCs (TI_MSP430_spi_USCIB0_5xx)
                                                   TI_TDC720x_SPIAutoIncReadReg (TI_MSP430_spi_USCIB0_5xx)
                                                   TI_TDC720x_SPIAutoIncWriteReg (TI_MSP430_spi_USCIB0_5xx)
                                                   TI_TDC720x_SPIByteReadReg (TI_MSP430_spi_USCIB0_5xx)
                                                   TI_TDC720x_SPIByteWriteReg (TI_MSP430_spi_USCIB0_5xx)
                                                   TI_TDC720x_SPILongReadReg (TI_MSP430_spi_USCIB0_5xx)
                                                   TI_TDC720x_SPISetup (TI_MSP430_spi_USCIB0_5xx)
                                                   handleHostCommand
                                                   handle_TDC720x_plus_mux (tdc720x_mode1_lt12ns)
                                                   handle_two_TDC720x (tdc720x_mode1_lt12ns)
                                                   main (main)
                                                   one_tdc_measure_results (tdc720x_measurement_control)
                                                   timer2_A0_init (timer_queue)
                                                   two_tdc_measure_results (tdc720x_measurement_control)
           ENTRY                   ADDRESS         REF BY
           =====                   =======         ======
           _A_PAOUT_L              0202 
           LOCAL                   ADDRESS         
           =====                   =======         
           PAOUT                   0202 
           PAOUT_H                 0203 
           PAOUT_L                 0202 
    -------------------------------------------------------------------------
DATA16_AN
  Relative segment, address: 020A - 020B (0x2 bytes), align: 0
  Segment part 2. ROOT        Intra module refs:   TIMER2_A0_ISR (timer_queue)
                                                   handleHostCommand
           ENTRY                   ADDRESS         REF BY
           =====                   =======         ======
           _A_PASEL_L              020A 
           LOCAL                   ADDRESS         
           =====                   =======         
           PASEL                   020A 
           PASEL_H                 020B 
           PASEL_L                 020A 
    -------------------------------------------------------------------------
DATA16_AN
  Relative segment, address: 0222 - 0223 (0x2 bytes), align: 0
  Segment part 3. ROOT        Intra module refs:   USBCommunicationTask (main)
                                                   handleHostCommand
                                                   main (main)
           ENTRY                   ADDRESS         REF BY
           =====                   =======         ======
           _A_PBOUT_L              0222 
           LOCAL                   ADDRESS         
           =====                   =======         
           PBOUT                   0222 
           PBOUT_H                 0223 
           PBOUT_L                 0222 
    -------------------------------------------------------------------------
DATA16_AN
  Relative segment, address: 0242 - 0243 (0x2 bytes), align: 0
  Segment part 4. ROOT        Intra module refs:   handleHostCommand
                                                   main (main)
           ENTRY                   ADDRESS         REF BY
           =====                   =======         ======
           _A_PCOUT_L              0242 
           LOCAL                   ADDRESS         
           =====                   =======         
           PCOUT                   0242 
           PCOUT_H                 0243 
           PCOUT_L                 0242 
    -------------------------------------------------------------------------
DATA16_AN
  Relative segment, address: 0262 - 0263 (0x2 bytes), align: 0
  Segment part 5. ROOT        Intra module refs:   handleHostCommand
                                                   handle_TDC720x_plus_mux (tdc720x_mode1_lt12ns)
                                                   main (main)
                                                   one_tdc_measure_results (tdc720x_measurement_control)
           ENTRY                   ADDRESS         REF BY
           =====                   =======         ======
           _A_PDOUT_L              0262 
           LOCAL                   ADDRESS         
           =====                   =======         
           PDOUT                   0262 
           PDOUT_H                 0263 
           PDOUT_L                 0262 
    -------------------------------------------------------------------------
DATA16_AN
  Relative segment, address: 0392 - 0393 (0x2 bytes), align: 0
  Segment part 6. ROOT        Intra module refs:   handleHostCommand
                                                   timer1_A0_init (timer_queue)
           ENTRY                   ADDRESS         REF BY
           =====                   =======         ======
           TA1CCR0                 0392 
    -------------------------------------------------------------------------
DATA16_AN
  Relative segment, address: 05E0 - 05E1 (0x2 bytes), align: 0
  Segment part 7. ROOT        Intra module refs:   TI_TDC720x_SPISetup (TI_MSP430_spi_USCIB0_5xx)
                                                   handleHostCommand
           ENTRY                   ADDRESS         REF BY
           =====                   =======         ======
           _A_UCB0CTLW0_L          05E0 
           LOCAL                   ADDRESS         
           =====                   =======         
           UCB0CTLW0               05E0 
           UCB0CTLW0_H             05E1 
           UCB0CTLW0_L             05E0 
    -------------------------------------------------------------------------
DATA16_AN
  Relative segment, address: 05E6 - 05E7 (0x2 bytes), align: 0
  Segment part 8. ROOT        Intra module refs:   TI_TDC720x_SPISetup (TI_MSP430_spi_USCIB0_5xx)
                                                   handleHostCommand
           ENTRY                   ADDRESS         REF BY
           =====                   =======         ======
           _A_UCB0BRW_L            05E6 
           LOCAL                   ADDRESS         
           =====                   =======         
           UCB0BRW                 05E6 
           UCB0BRW_H               05E7 
           UCB0BRW_L               05E6 
    -------------------------------------------------------------------------
DATA16_AN
  Relative segment, address: 0620 - 0621 (0x2 bytes), align: 0
  Segment part 9. ROOT        Intra module refs:   TI_TDC720x_SPIAllReadReg (TI_MSP430_spi_USCIB0_5xx)
                                                   TI_TDC720x_SPISetup (TI_MSP430_spi_USCIB0_5xx)
                                                   handleHostCommand
           ENTRY                   ADDRESS         REF BY
           =====                   =======         ======
           _A_UCB1CTLW0_L          0620 
           LOCAL                   ADDRESS         
           =====                   =======         
           UCB1CTLW0               0620 
           UCB1CTLW0_H             0621 
           UCB1CTLW0_L             0620 
    -------------------------------------------------------------------------
DATA16_AN
  Relative segment, address: 0626 - 0627 (0x2 bytes), align: 0
  Segment part 10. ROOT       Intra module refs:   handleHostCommand
           ENTRY                   ADDRESS         REF BY
           =====                   =======         ======
           _A_UCB1BRW_L            0626 
           LOCAL                   ADDRESS         
           =====                   =======         
           UCB1BRW                 0626 
           UCB1BRW_H               0627 
           UCB1BRW_L               0626 
    -------------------------------------------------------------------------
DATA16_Z
  Relative segment, address: 249E - 249E (0x1 bytes), align: 0
  Segment part 13.            Intra module refs:   handleHostCommand
           ENTRY                   ADDRESS         REF BY
           =====                   =======         ======
           TDC720x_UART_Stream     249E            USBCommunicationTask (main)
    -------------------------------------------------------------------------
DATA16_Z
  Relative segment, address: 249F - 249F (0x1 bytes), align: 0
  Segment part 14.            Intra module refs:   handleHostCommand
           ENTRY                   ADDRESS         REF BY
           =====                   =======         ======
           save_mode               249F 
    -------------------------------------------------------------------------
DATA16_Z
  Relative segment, address: 24A0 - 24C6 (0x27 bytes), align: 0
  Segment part 15.            Intra module refs:   handleHostCommand
           ENTRY                   ADDRESS         REF BY
           =====                   =======         ======
           all_data                24A0 
    -------------------------------------------------------------------------
DATA16_Z
  Relative segment, address: 24C7 - 24C7 (0x1 bytes), align: 0
  Segment part 16.            Intra module refs:   handleHostCommand
           ENTRY                   ADDRESS         REF BY
           =====                   =======         ======
           TDC720x_address         24C7 
    -------------------------------------------------------------------------
DATA16_Z
  Relative segment, address: 240E - 240F (0x2 bytes), align: 1
  Segment part 17.            Intra module refs:   handleHostCommand
           ENTRY                   ADDRESS         REF BY
           =====                   =======         ======
           save_default_timer_period
                                   240E 
    -------------------------------------------------------------------------
DATA16_Z
  Relative segment, address: 24C8 - 24C8 (0x1 bytes), align: 0
  Segment part 18.            Intra module refs:   handleHostCommand
           ENTRY                   ADDRESS         REF BY
           =====                   =======         ======
           save_timer_trig_freq    24C8 
    -------------------------------------------------------------------------
DATA16_Z
  Relative segment, address: 24C9 - 24C9 (0x1 bytes), align: 0
  Segment part 19.            Intra module refs:   handleHostCommand
           ENTRY                   ADDRESS         REF BY
           =====                   =======         ======
           save1_tdc7200_mode      24C9 
    -------------------------------------------------------------------------
DATA16_Z
  Relative segment, address: 24CA - 24CA (0x1 bytes), align: 0
  Segment part 20.            Intra module refs:   handleHostCommand
           ENTRY                   ADDRESS         REF BY
           =====                   =======         ======
           save2_tdc7200_mode      24CA 
    -------------------------------------------------------------------------
<CODE> 1 (was CODE)
  Relative segment, address: 4862 - 5203 (0x9a2 bytes), align: 1
  Segment part 23.
           ENTRY                   ADDRESS         REF BY
           =====                   =======         ======
           handleHostCommand       4862            USBCommunicationTask (main)
               calls direct and indirect
               CSTACK = 00000000 ( 00000016 )
    -------------------------------------------------------------------------
<CODE> 1 (was CODE)
  Relative segment, address: 9338 - 9339 (0x2 bytes), align: 1
  Segment part 22.            Intra module refs:   handleHostCommand
           ENTRY                   ADDRESS         REF BY
           =====                   =======         ======
           handle_reInit           9338 
               CSTACK = 00000000 ( 00000004 )
    -------------------------------------------------------------------------
<CODE> 1 (was CODE)
  Relative segment, address: 8AF2 - 8B27 (0x36 bytes), align: 1
  Segment part 21.            Intra module refs:   handleHostCommand
           ENTRY                   ADDRESS         REF BY
           =====                   =======         ======
           char2nibble             8AF2 
               CSTACK = 00000000 ( 00000004 )
    -------------------------------------------------------------------------
DATA16_C
  Relative segment, address: 4619 - 4627 (0xf bytes), align: 0
  Segment part 12.            Intra module refs:   handleHostCommand

    *************************************************************************

  FILE NAME : C:\Users\a0415888\Documents\pwd\GIT_REPOS\TDC7200\tdc7200evm_fw\Debug\Obj\ldopwr.r43
    *************************************************************************

  FILE NAME : C:\Users\a0415888\Documents\pwd\GIT_REPOS\TDC7200\tdc7200evm_fw\Debug\Obj\main.r43
  PROGRAM MODULE, NAME : main

  SEGMENTS IN THE MODULE
  ======================
DATA16_AN
  Relative segment, address: 0204 - 0205 (0x2 bytes), align: 0
  Segment part 2. ROOT        Intra module refs:   TI_TDC720x_SPISetup (TI_MSP430_spi_USCIB0_5xx)
                                                   main
                                                   timer2_A0_init (timer_queue)
           ENTRY                   ADDRESS         REF BY
           =====                   =======         ======
           _A_PADIR_L              0204 
           LOCAL                   ADDRESS         
           =====                   =======         
           PADIR                   0204 
           PADIR_H                 0205 
           PADIR_L                 0204 
    -------------------------------------------------------------------------
DATA16_AN
  Relative segment, address: 0206 - 0207 (0x2 bytes), align: 0
  Segment part 3. ROOT        Intra module refs:   main
           ENTRY                   ADDRESS         REF BY
           =====                   =======         ======
           _A_PAREN_L              0206 
           LOCAL                   ADDRESS         
           =====                   =======         
           PAREN                   0206 
           PAREN_H                 0207 
           PAREN_L                 0206 
    -------------------------------------------------------------------------
DATA16_AN
  Relative segment, address: 0218 - 0219 (0x2 bytes), align: 0
  Segment part 4. ROOT        Intra module refs:   main
           ENTRY                   ADDRESS         REF BY
           =====                   =======         ======
           _A_PAIES_L              0218 
           LOCAL                   ADDRESS         
           =====                   =======         
           PAIES                   0218 
           PAIES_H                 0219 
           PAIES_L                 0218 
    -------------------------------------------------------------------------
DATA16_AN
  Relative segment, address: 021C - 021D (0x2 bytes), align: 0
  Segment part 5. ROOT        Intra module refs:   main
           ENTRY                   ADDRESS         REF BY
           =====                   =======         ======
           _A_PAIFG_L              021C 
           LOCAL                   ADDRESS         
           =====                   =======         
           PAIFG                   021C 
           PAIFG_H                 021D 
           PAIFG_L                 021C 
    -------------------------------------------------------------------------
DATA16_AN
  Relative segment, address: 0224 - 0225 (0x2 bytes), align: 0
  Segment part 7. ROOT        Intra module refs:   InitUART (uart_commn)
                                                   TI_TDC720x_SPISetup (TI_MSP430_spi_USCIB0_5xx)
                                                   main
           ENTRY                   ADDRESS         REF BY
           =====                   =======         ======
           _A_PBDIR_L              0224 
           LOCAL                   ADDRESS         
           =====                   =======         
           PBDIR                   0224 
           PBDIR_H                 0225 
           PBDIR_L                 0224 
    -------------------------------------------------------------------------
DATA16_AN
  Relative segment, address: 0244 - 0245 (0x2 bytes), align: 0
  Segment part 9. ROOT        Intra module refs:   main
           ENTRY                   ADDRESS         REF BY
           =====                   =======         ======
           _A_PCDIR_L              0244 
           LOCAL                   ADDRESS         
           =====                   =======         
           PCDIR                   0244 
           PCDIR_H                 0245 
           PCDIR_L                 0244 
    -------------------------------------------------------------------------
DATA16_AN
  Relative segment, address: 024A - 024B (0x2 bytes), align: 0
  Segment part 10. ROOT       Intra module refs:   Init_Clock
           ENTRY                   ADDRESS         REF BY
           =====                   =======         ======
           _A_PCSEL_L              024A 
           LOCAL                   ADDRESS         
           =====                   =======         
           PCSEL                   024A 
           PCSEL_H                 024B 
           PCSEL_L                 024A 
    -------------------------------------------------------------------------
DATA16_AN
  Relative segment, address: 0264 - 0265 (0x2 bytes), align: 0
  Segment part 12. ROOT       Intra module refs:   main
           ENTRY                   ADDRESS         REF BY
           =====                   =======         ======
           _A_PDDIR_L              0264 
           LOCAL                   ADDRESS         
           =====                   =======         
           PDDIR                   0264 
           PDDIR_H                 0265 
           PDDIR_L                 0264 
    -------------------------------------------------------------------------
DATA16_AN
  Relative segment, address: 0198 - 0199 (0x2 bytes), align: 0
  Segment part 14. ROOT       Intra module refs:   UNMI_ISR
           ENTRY                   ADDRESS         REF BY
           =====                   =======         ======
           _A_SYSBERRIV_L          0198 
           LOCAL                   ADDRESS         
           =====                   =======         
           SYSBERRIV               0198 
           SYSBERRIV_H             0199 
           SYSBERRIV_L             0198 
    -------------------------------------------------------------------------
DATA16_AN
  Relative segment, address: 019A - 019B (0x2 bytes), align: 0
  Segment part 15. ROOT       Intra module refs:   UNMI_ISR
           ENTRY                   ADDRESS         REF BY
           =====                   =======         ======
           _A_SYSUNIV_L            019A 
           LOCAL                   ADDRESS         
           =====                   =======         
           SYSUNIV                 019A 
           SYSUNIV_H               019B 
           SYSUNIV_L               019A 
    -------------------------------------------------------------------------
DATA16_AN
  Relative segment, address: 0166 - 0167 (0x2 bytes), align: 0
  Segment part 19. ROOT       Intra module refs:   Init_Clock
                                                   USB_determineFreq (usb)
           ENTRY                   ADDRESS         REF BY
           =====                   =======         ======
           _A_UCSCTL3_L            0166 
           LOCAL                   ADDRESS         
           =====                   =======         
           UCSCTL3                 0166 
           UCSCTL3_H               0167 
           UCSCTL3_L               0166 
    -------------------------------------------------------------------------
DATA16_AN
  Relative segment, address: 015C - 015D (0x2 bytes), align: 0
  Segment part 23. ROOT       Intra module refs:   main
           ENTRY                   ADDRESS         REF BY
           =====                   =======         ======
           _A_WDTCTL_L             015C 
           LOCAL                   ADDRESS         
           =====                   =======         
           WDTCTL                  015C 
           WDTCTL_H                015D 
           WDTCTL_L                015C 
    -------------------------------------------------------------------------
DATA16_Z
  Relative segment, address: 24CB - 24CB (0x1 bytes), align: 0
  Segment part 26.            Intra module refs:   USBCommunicationTask
           ENTRY                   ADDRESS         REF BY
           =====                   =======         ======
           TDC720x_XYBufferReady   24CB            handle_TDC720x_plus_mux (tdc720x_mode1_lt12ns)
                                                   handle_two_TDC720x (tdc720x_mode1_lt12ns)
                                                   one_tdc_measure_results (tdc720x_measurement_control)
                                                   two_tdc_measure_results (tdc720x_measurement_control)
    -------------------------------------------------------------------------
DATA16_Z
  Relative segment, address: 24CC - 24CC (0x1 bytes), align: 0
  Segment part 27.            Intra module refs:   USBCommunicationTask
           ENTRY                   ADDRESS         REF BY
           =====                   =======         ======
           TDC720x_PQBufferReady   24CC            handle_TDC720x_plus_mux (tdc720x_mode1_lt12ns)
                                                   handle_two_TDC720x (tdc720x_mode1_lt12ns)
                                                   two_tdc_measure_results (tdc720x_measurement_control)
    -------------------------------------------------------------------------
DATA16_Z
  Relative segment, address: 24CD - 24CD (0x1 bytes), align: 0
  Segment part 28.            Intra module refs:   USBCommunicationTask
           ENTRY                   ADDRESS         REF BY
           =====                   =======         ======
           bCDCDataReceived_event
                                   24CD            USBCDC_handleDataReceived (usbEventHandling)
    -------------------------------------------------------------------------
DATA16_Z
  Relative segment, address: 2410 - 2411 (0x2 bytes), align: 1
  Segment part 29.            Intra module refs:   USBCommunicationTask
           ENTRY                   ADDRESS         REF BY
           =====                   =======         ======
           w                       2410 
    -------------------------------------------------------------------------
DATA16_Z
  Relative segment, address: 24CE - 24F4 (0x27 bytes), align: 0
  Segment part 30.            Intra module refs:   Segment part 33
           ENTRY                   ADDRESS         REF BY
           =====                   =======         ======
           bufferX                 24CE            handle_TDC720x_plus_mux (tdc720x_mode1_lt12ns)
                                                   handle_two_TDC720x (tdc720x_mode1_lt12ns)
                                                   one_tdc_measure_results (tdc720x_measurement_control)
                                                   two_tdc_measure_results (tdc720x_measurement_control)
    -------------------------------------------------------------------------
DATA16_Z
  Relative segment, address: 24F5 - 251B (0x27 bytes), align: 0
  Segment part 31.
           ENTRY                   ADDRESS         REF BY
           =====                   =======         ======
           bufferY                 24F5            handle_TDC720x_plus_mux (tdc720x_mode1_lt12ns)
                                                   handle_two_TDC720x (tdc720x_mode1_lt12ns)
                                                   one_tdc_measure_results (tdc720x_measurement_control)
                                                   two_tdc_measure_results (tdc720x_measurement_control)
    -------------------------------------------------------------------------
DATA16_I
  Relative segment, address: 2400 - 2401 (0x2 bytes), align: 1
  Segment part 32.
           ENTRY                   ADDRESS         REF BY
           =====                   =======         ======
           mbuf                    2400            handle_TDC720x_plus_mux (tdc720x_mode1_lt12ns)
                                                   handle_two_TDC720x (tdc720x_mode1_lt12ns)
                                                   one_tdc_measure_results (tdc720x_measurement_control)
                                                   two_tdc_measure_results (tdc720x_measurement_control)
    -------------------------------------------------------------------------
DATA16_Z
  Relative segment, address: 2412 - 2413 (0x2 bytes), align: 1
  Segment part 34.            Intra module refs:   USBCommunicationTask
           ENTRY                   ADDRESS         REF BY
           =====                   =======         ======
           ubuf                    2412            handle_TDC720x_plus_mux (tdc720x_mode1_lt12ns)
                                                   handle_two_TDC720x (tdc720x_mode1_lt12ns)
                                                   one_tdc_measure_results (tdc720x_measurement_control)
                                                   two_tdc_measure_results (tdc720x_measurement_control)
    -------------------------------------------------------------------------
DATA16_Z
  Relative segment, address: 251C - 2542 (0x27 bytes), align: 0
  Segment part 35.            Intra module refs:   Segment part 38
           ENTRY                   ADDRESS         REF BY
           =====                   =======         ======
           bufferP                 251C            handle_TDC720x_plus_mux (tdc720x_mode1_lt12ns)
                                                   handle_two_TDC720x (tdc720x_mode1_lt12ns)
                                                   two_tdc_measure_results (tdc720x_measurement_control)
    -------------------------------------------------------------------------
DATA16_Z
  Relative segment, address: 2543 - 2569 (0x27 bytes), align: 0
  Segment part 36.
           ENTRY                   ADDRESS         REF BY
           =====                   =======         ======
           bufferQ                 2543            handle_TDC720x_plus_mux (tdc720x_mode1_lt12ns)
                                                   handle_two_TDC720x (tdc720x_mode1_lt12ns)
                                                   two_tdc_measure_results (tdc720x_measurement_control)
    -------------------------------------------------------------------------
DATA16_I
  Relative segment, address: 2402 - 2403 (0x2 bytes), align: 1
  Segment part 37.
           ENTRY                   ADDRESS         REF BY
           =====                   =======         ======
           nbuf                    2402            handle_TDC720x_plus_mux (tdc720x_mode1_lt12ns)
                                                   handle_two_TDC720x (tdc720x_mode1_lt12ns)
                                                   two_tdc_measure_results (tdc720x_measurement_control)
    -------------------------------------------------------------------------
DATA16_Z
  Relative segment, address: 2414 - 2415 (0x2 bytes), align: 1
  Segment part 39.            Intra module refs:   USBCommunicationTask
           ENTRY                   ADDRESS         REF BY
           =====                   =======         ======
           vbuf                    2414            handle_TDC720x_plus_mux (tdc720x_mode1_lt12ns)
                                                   handle_two_TDC720x (tdc720x_mode1_lt12ns)
                                                   two_tdc_measure_results (tdc720x_measurement_control)
    -------------------------------------------------------------------------
DATA16_Z
  Relative segment, address: 256A - 2589 (0x20 bytes), align: 0
  Segment part 40.            Intra module refs:   USBCommunicationTask
           ENTRY                   ADDRESS         REF BY
           =====                   =======         ======
           cmdResponseString       256A 
    -------------------------------------------------------------------------
DATA16_Z
  Relative segment, address: 258A - 258A (0x1 bytes), align: 0
  Segment part 41.            Intra module refs:   USBCommunicationTask
           ENTRY                   ADDRESS         REF BY
           =====                   =======         ======
           single_shot_measure_state
                                   258A            handleHostCommand (host_interface)
                                                   tdc_trigger_measure (timer_queue)
    -------------------------------------------------------------------------
DATA16_Z
  Relative segment, address: 258B - 258B (0x1 bytes), align: 0
  Segment part 42.            Intra module refs:   USBCommunicationTask
           ENTRY                   ADDRESS         REF BY
           =====                   =======         ======
           tof_graph_state         258B            handleHostCommand (host_interface)
                                                   tdc_trigger_measure (timer_queue)
    -------------------------------------------------------------------------
DATA16_Z
  Relative segment, address: 258C - 258C (0x1 bytes), align: 0
  Segment part 43.
           ENTRY                   ADDRESS         REF BY
           =====                   =======         ======
           graph_delay_sweep_state
                                   258C            handleHostCommand (host_interface)
    -------------------------------------------------------------------------
DATA16_Z
  Relative segment, address: 258D - 258D (0x1 bytes), align: 0
  Segment part 44.
           ENTRY                   ADDRESS         REF BY
           =====                   =======         ======
           double_resolution       258D            handleHostCommand (host_interface)
    -------------------------------------------------------------------------
DATA16_Z
  Relative segment, address: 258E - 258E (0x1 bytes), align: 0
  Segment part 45.
           ENTRY                   ADDRESS         REF BY
           =====                   =======         ======
           current_tdc             258E            handleHostCommand (host_interface)
                                                   one_tdc_measure_results (tdc720x_measurement_control)
    -------------------------------------------------------------------------
DATA16_I
  Relative segment, address: 240C - 240C (0x1 bytes), align: 0
  Segment part 46.            Intra module refs:   main
           ENTRY                   ADDRESS         REF BY
           =====                   =======         ======
           TDC720xEVM_Device       240C            handleHostCommand (host_interface)
    -------------------------------------------------------------------------
DATA16_Z
  Relative segment, address: 2416 - 2419 (0x4 bytes), align: 1
  Segment part 48.            Intra module refs:   USBCommunicationTask
           ENTRY                   ADDRESS         REF BY
           =====                   =======         ======
           err_count               2416 
    -------------------------------------------------------------------------
<CODE> 1 (was CODE)
  Relative segment, address: 6ECA - 6FA3 (0xda bytes), align: 1
  Segment part 53.
           ENTRY                   ADDRESS         REF BY
           =====                   =======         ======
           main                    6ECA            Segment part 26 (?cstart)
               calls direct
               CSTACK = 00000000 ( 00000004 )
    -------------------------------------------------------------------------
<CODE> 1 (was CODE)
  Relative segment, address: 8CF8 - 8D23 (0x2c bytes), align: 1
  Segment part 52.            Intra module refs:   main
           ENTRY                   ADDRESS         REF BY
           =====                   =======         ======
           InitMCU                 8CF8 
               calls direct
               CSTACK = 00000000 ( 00000004 )
    -------------------------------------------------------------------------
<CODE> 1 (was CODE)
  Relative segment, address: 643E - 65AB (0x16e bytes), align: 1
  Segment part 51.            Intra module refs:   main
           ENTRY                   ADDRESS         REF BY
           =====                   =======         ======
           USBCommunicationTask    643E 
               calls direct
               CSTACK = 00000000 ( 00000010 )
    -------------------------------------------------------------------------
<CODE> 1 (was CODE)
  Relative segment, address: 7074 - 713D (0xca bytes), align: 1
  Segment part 50.            Intra module refs:   InitMCU
           ENTRY                   ADDRESS         REF BY
           =====                   =======         ======
           Init_Clock              7074 
               CSTACK = 00000000 ( 00000004 )
    -------------------------------------------------------------------------
ISR_CODE
  Relative segment, address: 46B8 - 46ED (0x36 bytes), align: 1
  Segment part 54.            Intra module refs:   UNMI_ISR::??INTVEC 122
           ENTRY                   ADDRESS         REF BY
           =====                   =======         ======
           UNMI_ISR                46B8 
               interrupt function
               calls direct
               CSTACK = 00000000 ( 0000000C )
    -------------------------------------------------------------------------
<CODE> 1 (was CODE)
  Relative segment, address: 7E3A - 7EB5 (0x7c bytes), align: 1
  Segment part 49.            Intra module refs:   main
           ENTRY                   ADDRESS         REF BY
           =====                   =======         ======
           TI_TDC720x_reg_init     7E3A            handleHostCommand (host_interface)
               calls direct
               CSTACK = 00000000 ( 00000006 )
    -------------------------------------------------------------------------
INTVEC
  Common segment, address: FF80 - FFFB (0x7c bytes), align: 1
  Segment part 24. ROOT 
           ENTRY                   ADDRESS         REF BY
           =====                   =======         ======
           UNMI_ISR::??INTVEC 122
                                   FFFA 
    -------------------------------------------------------------------------
DATA16_ID
  Relative segment, address: 4682 - 4683 (0x2 bytes), align: 1
  Segment part 33.            Intra module refs:   mbuf
    -------------------------------------------------------------------------
DATA16_ID
  Relative segment, address: 4684 - 4685 (0x2 bytes), align: 1
  Segment part 38.            Intra module refs:   nbuf
    -------------------------------------------------------------------------
DATA16_ID
  Relative segment, address: 468E - 468E (0x1 bytes), align: 0
  Segment part 47.            Intra module refs:   TDC720xEVM_Device

    *************************************************************************

  FILE NAME : C:\Users\a0415888\Documents\pwd\GIT_REPOS\TDC7200\tdc7200evm_fw\Debug\Obj\mpy32.r43
    *************************************************************************

  FILE NAME : C:\Users\a0415888\Documents\pwd\GIT_REPOS\TDC7200\tdc7200evm_fw\Debug\Obj\pmap.r43
    *************************************************************************

  FILE NAME : C:\Users\a0415888\Documents\pwd\GIT_REPOS\TDC7200\tdc7200evm_fw\Debug\Obj\pmm.r43
    *************************************************************************

  FILE NAME : C:\Users\a0415888\Documents\pwd\GIT_REPOS\TDC7200\tdc7200evm_fw\Debug\Obj\ram.r43
    *************************************************************************

  FILE NAME : C:\Users\a0415888\Documents\pwd\GIT_REPOS\TDC7200\tdc7200evm_fw\Debug\Obj\ref.r43
    *************************************************************************

  FILE NAME : C:\Users\a0415888\Documents\pwd\GIT_REPOS\TDC7200\tdc7200evm_fw\Debug\Obj\rtc_a.r43
    *************************************************************************

  FILE NAME : C:\Users\a0415888\Documents\pwd\GIT_REPOS\TDC7200\tdc7200evm_fw\Debug\Obj\rtc_b.r43
    *************************************************************************

  FILE NAME : C:\Users\a0415888\Documents\pwd\GIT_REPOS\TDC7200\tdc7200evm_fw\Debug\Obj\rtc_c.r43
    *************************************************************************

  FILE NAME : C:\Users\a0415888\Documents\pwd\GIT_REPOS\TDC7200\tdc7200evm_fw\Debug\Obj\sd24_b.r43
    *************************************************************************

  FILE NAME : C:\Users\a0415888\Documents\pwd\GIT_REPOS\TDC7200\tdc7200evm_fw\Debug\Obj\sfr.r43
    *************************************************************************

  FILE NAME : C:\Users\a0415888\Documents\pwd\GIT_REPOS\TDC7200\tdc7200evm_fw\Debug\Obj\sysctl.r43
    *************************************************************************

  FILE NAME : C:\Users\a0415888\Documents\pwd\GIT_REPOS\TDC7200\tdc7200evm_fw\Debug\Obj\tdc720x_calculation.r43
  PROGRAM MODULE, NAME : tdc720x_calculation

  SEGMENTS IN THE MODULE
  ======================
DATA16_I
  Relative segment, address: 2404 - 2407 (0x4 bytes), align: 1
  Segment part 4.             Intra module refs:   TDC720x_normlsb
                                                   TDC720x_start2stopn
           ENTRY                   ADDRESS         REF BY
           =====                   =======         ======
           tdc_clk_period          2404            handleHostCommand (host_interface)
    -------------------------------------------------------------------------
DATA16_Z
  Relative segment, address: 241A - 242D (0x14 bytes), align: 1
  Segment part 6.             Intra module refs:   TDC720x_start2stopn
                                                   print_start2stopn
           ENTRY                   ADDRESS         REF BY
           =====                   =======         ======
           start2stop              241A 
    -------------------------------------------------------------------------
DATA16_Z
  Relative segment, address: 258F - 260E (0x80 bytes), align: 0
  Segment part 7.             Intra module refs:   print_start2stopn
           ENTRY                   ADDRESS         REF BY
           =====                   =======         ======
           outString               258F            handleHostCommand (host_interface)
    -------------------------------------------------------------------------
DATA16_Z
  Relative segment, address: 242E - 2461 (0x34 bytes), align: 1
  Segment part 8.             Intra module refs:   TDC720x_build_mreg
                                                   TDC720x_normlsb
                                                   TDC720x_start2stopn
           ENTRY                   ADDRESS         REF BY
           =====                   =======         ======
           meas_result_regrs       242E 
    -------------------------------------------------------------------------
DATA16_Z
  Relative segment, address: 2462 - 2465 (0x4 bytes), align: 1
  Segment part 9.             Intra module refs:   TDC720x_normlsb
                                                   TDC720x_start2stopn
           ENTRY                   ADDRESS         REF BY
           =====                   =======         ======
           norm_lsb                2462 
    -------------------------------------------------------------------------
DATA16_Z
  Relative segment, address: 2466 - 2469 (0x4 bytes), align: 1
  Segment part 10.            Intra module refs:   TDC720x_normlsb
           ENTRY                   ADDRESS         REF BY
           =====                   =======         ======
           ccnt                    2466 
    -------------------------------------------------------------------------
<CODE> 1 (was CODE)
  Relative segment, address: 8FBE - 8FD3 (0x16 bytes), align: 1
  Segment part 15.
           ENTRY                   ADDRESS         REF BY
           =====                   =======         ======
           TDC720x_calc            8FBE            USBCommunicationTask (main)
               calls direct
               CSTACK = 00000000 ( 00000006 )
    -------------------------------------------------------------------------
<CODE> 1 (was CODE)
  Relative segment, address: 82AA - 830D (0x64 bytes), align: 1
  Segment part 14.            Intra module refs:   TDC720x_calc
           ENTRY                   ADDRESS         REF BY
           =====                   =======         ======
           print_start2stopn       82AA 
               calls direct
               CSTACK = 00000000 ( 0000000C )
    -------------------------------------------------------------------------
<CODE> 1 (was CODE)
  Relative segment, address: 7FAA - 8021 (0x78 bytes), align: 1
  Segment part 13.            Intra module refs:   TDC720x_calc
           ENTRY                   ADDRESS         REF BY
           =====                   =======         ======
           TDC720x_start2stopn     7FAA 
               calls direct
               CSTACK = 00000000 ( 00000010 )
    -------------------------------------------------------------------------
<CODE> 1 (was CODE)
  Relative segment, address: 7A0C - 7A9B (0x90 bytes), align: 1
  Segment part 12.            Intra module refs:   TDC720x_start2stopn
           ENTRY                   ADDRESS         REF BY
           =====                   =======         ======
           TDC720x_normlsb         7A0C 
               calls direct
               CSTACK = 00000000 ( 00000008 )
    -------------------------------------------------------------------------
<CODE> 1 (was CODE)
  Relative segment, address: 8022 - 8093 (0x72 bytes), align: 1
  Segment part 11.            Intra module refs:   TDC720x_calc
           ENTRY                   ADDRESS         REF BY
           =====                   =======         ======
           TDC720x_build_mreg      8022 
               CSTACK = 00000000 ( 00000008 )
    -------------------------------------------------------------------------
DATA16_ID
  Relative segment, address: 4686 - 4689 (0x4 bytes), align: 1
  Segment part 5.             Intra module refs:   tdc_clk_period
    -------------------------------------------------------------------------
DATA16_C
  Relative segment, address: 4628 - 4644 (0x1d bytes), align: 0
  Segment part 2.             Intra module refs:   print_start2stopn
    -------------------------------------------------------------------------
DATA16_C
  Relative segment, address: 4645 - 4648 (0x4 bytes), align: 0
  Segment part 3.             Intra module refs:   print_start2stopn

    *************************************************************************

  FILE NAME : C:\Users\a0415888\Documents\pwd\GIT_REPOS\TDC7200\tdc7200evm_fw\Debug\Obj\tdc720x_measurement_control.r43
  PROGRAM MODULE, NAME : tdc720x_measurement_control

  SEGMENTS IN THE MODULE
  ======================
DATA16_Z
  Relative segment, address: 260F - 260F (0x1 bytes), align: 0
  Segment part 4.             Intra module refs:   two_tdc_measure_results
           ENTRY                   ADDRESS         REF BY
           =====                   =======         ======
           TDC720x_Parallel_Read   260F            TI_TDC720x_SPIAllReadReg (TI_MSP430_spi_USCIB0_5xx)
                                                   TI_TDC720x_SPIAutoIncReadReg (TI_MSP430_spi_USCIB0_5xx)
                                                   TI_TDC720x_SPIByteReadReg (TI_MSP430_spi_USCIB0_5xx)
                                                   TI_TDC720x_SPILongReadReg (TI_MSP430_spi_USCIB0_5xx)
                                                   handleHostCommand (host_interface)
    -------------------------------------------------------------------------
<CODE> 1 (was CODE)
  Relative segment, address: 7CC0 - 7D3D (0x7e bytes), align: 1
  Segment part 6.
           ENTRY                   ADDRESS         REF BY
           =====                   =======         ======
           one_tdc_measure_results
                                   7CC0            tdc_trigger_measure (timer_queue)
               calls direct
               CSTACK = 00000000 ( 00000004 )
    -------------------------------------------------------------------------
<CODE> 1 (was CODE)
  Relative segment, address: 72CA - 7389 (0xc0 bytes), align: 1
  Segment part 5.
           ENTRY                   ADDRESS         REF BY
           =====                   =======         ======
           two_tdc_measure_results
                                   72CA            tdc_trigger_measure (timer_queue)
               calls direct
               CSTACK = 00000000 ( 00000008 )

    *************************************************************************

  FILE NAME : C:\Users\a0415888\Documents\pwd\GIT_REPOS\TDC7200\tdc7200evm_fw\Debug\Obj\tdc720x_mode1_lt12ns.r43
  PROGRAM MODULE, NAME : tdc720x_mode1_lt12ns

  SEGMENTS IN THE MODULE
  ======================
<CODE> 1 (was CODE)
  Relative segment, address: 8F92 - 8FA7 (0x16 bytes), align: 1
  Segment part 6.
           ENTRY                   ADDRESS         REF BY
           =====                   =======         ======
           TDC720x_mode1_lt12ns    8F92            tdc_trigger_measure (timer_queue)
               calls direct
               CSTACK = 00000000 ( 00000004 )
    -------------------------------------------------------------------------
<CODE> 1 (was CODE)
  Relative segment, address: 738A - 7435 (0xac bytes), align: 1
  Segment part 5.             Intra module refs:   TDC720x_mode1_lt12ns
           ENTRY                   ADDRESS         REF BY
           =====                   =======         ======
           handle_two_TDC720x      738A 
               calls direct
               CSTACK = 00000000 ( 00000008 )
    -------------------------------------------------------------------------
<CODE> 1 (was CODE)
  Relative segment, address: 6FA4 - 7073 (0xd0 bytes), align: 1
  Segment part 4.             Intra module refs:   TDC720x_mode1_lt12ns
           ENTRY                   ADDRESS         REF BY
           =====                   =======         ======
           handle_TDC720x_plus_mux
                                   6FA4 
               calls direct
               CSTACK = 00000000 ( 00000006 )

    *************************************************************************

  FILE NAME : C:\Users\a0415888\Documents\pwd\GIT_REPOS\TDC7200\tdc7200evm_fw\Debug\Obj\tec.r43
    *************************************************************************

  FILE NAME : C:\Users\a0415888\Documents\pwd\GIT_REPOS\TDC7200\tdc7200evm_fw\Debug\Obj\TI_MSP430_spi_USCIB0_5xx.r43
  PROGRAM MODULE, NAME : TI_MSP430_spi_USCIB0_5xx

  SEGMENTS IN THE MODULE
  ======================
DATA16_AN
  Relative segment, address: 022A - 022B (0x2 bytes), align: 0
  Segment part 4. ROOT        Intra module refs:   InitUART (uart_commn)
                                                   TI_TDC720x_SPISetup
           ENTRY                   ADDRESS         REF BY
           =====                   =======         ======
           _A_PBSEL_L              022A 
           LOCAL                   ADDRESS         
           =====                   =======         
           PBSEL                   022A 
           PBSEL_H                 022B 
           PBSEL_L                 022A 
    -------------------------------------------------------------------------
DATA16_AN
  Relative segment, address: 05EA - 05EA (0x1 bytes), align: 0
  Segment part 7. ROOT        Intra module refs:   TI_TDC720x_SPIAllReadReg
                                                   TI_TDC720x_SPIAllReadReg_BothTDCs
                                                   TI_TDC720x_SPIAutoIncReadReg
                                                   TI_TDC720x_SPIAutoIncWriteReg
                                                   TI_TDC720x_SPIByteReadReg
                                                   TI_TDC720x_SPIByteWriteReg
                                                   TI_TDC720x_SPILongReadReg
           ENTRY                   ADDRESS         REF BY
           =====                   =======         ======
           UCB0STAT                05EA 
    -------------------------------------------------------------------------
DATA16_AN
  Relative segment, address: 05EC - 05EC (0x1 bytes), align: 0
  Segment part 8. ROOT        Intra module refs:   TI_TDC720x_SPIAllReadReg
                                                   TI_TDC720x_SPIAllReadReg_BothTDCs
                                                   TI_TDC720x_SPIAutoIncReadReg
                                                   TI_TDC720x_SPIByteReadReg
                                                   TI_TDC720x_SPILongReadReg
           ENTRY                   ADDRESS         REF BY
           =====                   =======         ======
           UCB0RXBUF               05EC 
    -------------------------------------------------------------------------
DATA16_AN
  Relative segment, address: 05EE - 05EE (0x1 bytes), align: 0
  Segment part 9. ROOT        Intra module refs:   TI_TDC720x_SPIAllReadReg
                                                   TI_TDC720x_SPIAllReadReg_BothTDCs
                                                   TI_TDC720x_SPIAutoIncReadReg
                                                   TI_TDC720x_SPIAutoIncWriteReg
                                                   TI_TDC720x_SPIByteReadReg
                                                   TI_TDC720x_SPIByteWriteReg
                                                   TI_TDC720x_SPILongReadReg
           ENTRY                   ADDRESS         REF BY
           =====                   =======         ======
           UCB0TXBUF               05EE 
    -------------------------------------------------------------------------
DATA16_AN
  Relative segment, address: 05FC - 05FD (0x2 bytes), align: 0
  Segment part 10. ROOT       Intra module refs:   TI_TDC720x_SPIAllReadReg
                                                   TI_TDC720x_SPIAllReadReg_BothTDCs
                                                   TI_TDC720x_SPIAutoIncReadReg
                                                   TI_TDC720x_SPIAutoIncWriteReg
                                                   TI_TDC720x_SPIByteReadReg
                                                   TI_TDC720x_SPIByteWriteReg
                                                   TI_TDC720x_SPILongReadReg
           ENTRY                   ADDRESS         REF BY
           =====                   =======         ======
           _A_UCB0ICTL_L           05FC 
           LOCAL                   ADDRESS         
           =====                   =======         
           UCB0ICTL                05FC 
           UCB0ICTL_H              05FD 
           UCB0ICTL_L              05FC 
    -------------------------------------------------------------------------
DATA16_AN
  Relative segment, address: 062A - 062A (0x1 bytes), align: 0
  Segment part 12. ROOT       Intra module refs:   TI_TDC720x_SPIByteReadReg
           ENTRY                   ADDRESS         REF BY
           =====                   =======         ======
           UCB1STAT                062A 
    -------------------------------------------------------------------------
DATA16_AN
  Relative segment, address: 062C - 062C (0x1 bytes), align: 0
  Segment part 13. ROOT       Intra module refs:   TI_TDC720x_SPIAllReadReg
                                                   TI_TDC720x_SPIAllReadReg_BothTDCs
                                                   TI_TDC720x_SPIAutoIncReadReg
                                                   TI_TDC720x_SPIByteReadReg
                                                   TI_TDC720x_SPILongReadReg
           ENTRY                   ADDRESS         REF BY
           =====                   =======         ======
           UCB1RXBUF               062C 
    -------------------------------------------------------------------------
DATA16_AN
  Relative segment, address: 063C - 063D (0x2 bytes), align: 0
  Segment part 14. ROOT       Intra module refs:   TI_TDC720x_SPIAllReadReg
                                                   TI_TDC720x_SPIAllReadReg_BothTDCs
                                                   TI_TDC720x_SPIAutoIncReadReg
                                                   TI_TDC720x_SPILongReadReg
           ENTRY                   ADDRESS         REF BY
           =====                   =======         ======
           _A_UCB1ICTL_L           063C 
           LOCAL                   ADDRESS         
           =====                   =======         
           UCB1ICTL                063C 
           UCB1ICTL_H              063D 
           UCB1ICTL_L              063C 
    -------------------------------------------------------------------------
<CODE> 1 (was CODE)
  Relative segment, address: 8242 - 82A9 (0x68 bytes), align: 1
  Segment part 24.
           ENTRY                   ADDRESS         REF BY
           =====                   =======         ======
           TI_TDC720x_SPISetup     8242            main (main)
               CSTACK = 00000000 ( 00000004 )
    -------------------------------------------------------------------------
<CODE> 1 (was CODE)
  Relative segment, address: 87C2 - 8809 (0x48 bytes), align: 1
  Segment part 23.
           ENTRY                   ADDRESS         REF BY
           =====                   =======         ======
           TI_TDC720x_SPIByteWriteReg
                                   87C2            TI_TDC720x_reg_init (main)
                                                   handleHostCommand (host_interface)
                                                   handle_TDC720x_plus_mux (tdc720x_mode1_lt12ns)
                                                   handle_two_TDC720x (tdc720x_mode1_lt12ns)
                                                   one_tdc_measure_results (tdc720x_measurement_control)
                                                   two_tdc_measure_results (tdc720x_measurement_control)
               CSTACK = 00000000 ( 00000004 )
    -------------------------------------------------------------------------
<CODE> 1 (was CODE)
  Relative segment, address: 8370 - 83CF (0x60 bytes), align: 1
  Segment part 22.
           ENTRY                   ADDRESS         REF BY
           =====                   =======         ======
           TI_TDC720x_SPIByteReadReg
                                   8370            TDC720x_normlsb (tdc720x_calculation)
                                                   handleHostCommand (host_interface)
                                                   handle_TDC720x_plus_mux (tdc720x_mode1_lt12ns)
                                                   handle_two_TDC720x (tdc720x_mode1_lt12ns)
                                                   one_tdc_measure_results (tdc720x_measurement_control)
                                                   two_tdc_measure_results (tdc720x_measurement_control)
               CSTACK = 00000000 ( 00000004 )
    -------------------------------------------------------------------------
<CODE> 1 (was CODE)
  Relative segment, address: 84EA - 8541 (0x58 bytes), align: 1
  Segment part 21.
           ENTRY                   ADDRESS         REF BY
           =====                   =======         ======
           TI_TDC720x_SPIAutoIncWriteReg
                                   84EA            handleHostCommand (host_interface)
               CSTACK = 00000000 ( 00000004 )
    -------------------------------------------------------------------------
<CODE> 1 (was CODE)
  Relative segment, address: 7DBC - 7E39 (0x7e bytes), align: 1
  Segment part 20.
           ENTRY                   ADDRESS         REF BY
           =====                   =======         ======
           TI_TDC720x_SPIAutoIncReadReg
                                   7DBC            handleHostCommand (host_interface)
               CSTACK = 00000000 ( 00000006 )
    -------------------------------------------------------------------------
<CODE> 1 (was CODE)
  Relative segment, address: 7B2A - 7BB5 (0x8c bytes), align: 1
  Segment part 19.
           ENTRY                   ADDRESS         REF BY
           =====                   =======         ======
           TI_TDC720x_SPIAllReadReg
                                   7B2A            handle_TDC720x_plus_mux (tdc720x_mode1_lt12ns)
                                                   handle_two_TDC720x (tdc720x_mode1_lt12ns)
                                                   one_tdc_measure_results (tdc720x_measurement_control)
                                                   two_tdc_measure_results (tdc720x_measurement_control)
               CSTACK = 00000000 ( 00000004 )
    -------------------------------------------------------------------------
<CODE> 1 (was CODE)
  Relative segment, address: 6D06 - 6DED (0xe8 bytes), align: 1
  Segment part 18.
           ENTRY                   ADDRESS         REF BY
           =====                   =======         ======
           TI_TDC720x_SPILongReadReg
                                   6D06            handleHostCommand (host_interface)
               CSTACK = 00000000 ( 00000008 )
    -------------------------------------------------------------------------
<CODE> 1 (was CODE)
  Relative segment, address: 83D0 - 842D (0x5e bytes), align: 1
  Segment part 16.
           ENTRY                   ADDRESS         REF BY
           =====                   =======         ======
           TI_TDC720x_SPIAllReadReg_BothTDCs
                                   83D0            two_tdc_measure_results (tdc720x_measurement_control)
               CSTACK = 00000000 ( 00000004 )

    *************************************************************************

  FILE NAME : C:\Users\a0415888\Documents\pwd\GIT_REPOS\TDC7200\tdc7200evm_fw\Debug\Obj\timer_a.r43
    *************************************************************************

  FILE NAME : C:\Users\a0415888\Documents\pwd\GIT_REPOS\TDC7200\tdc7200evm_fw\Debug\Obj\timer_b.r43
    *************************************************************************

  FILE NAME : C:\Users\a0415888\Documents\pwd\GIT_REPOS\TDC7200\tdc7200evm_fw\Debug\Obj\timer_d.r43
    *************************************************************************

  FILE NAME : C:\Users\a0415888\Documents\pwd\GIT_REPOS\TDC7200\tdc7200evm_fw\Debug\Obj\timer_queue.r43
  PROGRAM MODULE, NAME : timer_queue

  SEGMENTS IN THE MODULE
  ======================
DATA16_AN
  Relative segment, address: 0200 - 0201 (0x2 bytes), align: 0
  Segment part 1. ROOT        Intra module refs:   wait_on_intb_pin
           ENTRY                   ADDRESS         REF BY
           =====                   =======         ======
           _A_PAIN_L               0200 
           LOCAL                   ADDRESS         
           =====                   =======         
           PAIN                    0200 
           PAIN_H                  0201 
           PAIN_L                  0200 
    -------------------------------------------------------------------------
DATA16_AN
  Relative segment, address: 0208 - 0209 (0x2 bytes), align: 0
  Segment part 4. ROOT        Intra module refs:   timer2_A0_init
           ENTRY                   ADDRESS         REF BY
           =====                   =======         ======
           _A_PADS_L               0208 
           LOCAL                   ADDRESS         
           =====                   =======         
           PADS                    0208 
           PADS_H                  0209 
           PADS_L                  0208 
    -------------------------------------------------------------------------
DATA16_AN
  Relative segment, address: 0340 - 0341 (0x2 bytes), align: 0
  Segment part 6. ROOT 
           ENTRY                   ADDRESS         REF BY
           =====                   =======         ======
           TA0CTL                  0340 
    -------------------------------------------------------------------------
DATA16_AN
  Relative segment, address: 0342 - 0343 (0x2 bytes), align: 0
  Segment part 7. ROOT 
           ENTRY                   ADDRESS         REF BY
           =====                   =======         ======
           TA0CCTL0                0342 
    -------------------------------------------------------------------------
DATA16_AN
  Relative segment, address: 0352 - 0353 (0x2 bytes), align: 0
  Segment part 8. ROOT 
           ENTRY                   ADDRESS         REF BY
           =====                   =======         ======
           TA0CCR0                 0352 
    -------------------------------------------------------------------------
DATA16_AN
  Relative segment, address: 0380 - 0381 (0x2 bytes), align: 0
  Segment part 9. ROOT        Intra module refs:   timer1_A0_init
           ENTRY                   ADDRESS         REF BY
           =====                   =======         ======
           TA1CTL                  0380 
    -------------------------------------------------------------------------
DATA16_AN
  Relative segment, address: 0382 - 0383 (0x2 bytes), align: 0
  Segment part 10. ROOT       Intra module refs:   timer1_A0_init
           ENTRY                   ADDRESS         REF BY
           =====                   =======         ======
           TA1CCTL0                0382 
    -------------------------------------------------------------------------
DATA16_AN
  Relative segment, address: 03A0 - 03A1 (0x2 bytes), align: 0
  Segment part 12. ROOT       Intra module refs:   timer1_A0_init
           ENTRY                   ADDRESS         REF BY
           =====                   =======         ======
           TA1EX0                  03A0 
    -------------------------------------------------------------------------
DATA16_AN
  Relative segment, address: 0400 - 0401 (0x2 bytes), align: 0
  Segment part 13. ROOT       Intra module refs:   TIMER2_A0_ISR
                                                   timer2_A0_init
           ENTRY                   ADDRESS         REF BY
           =====                   =======         ======
           TA2CTL                  0400 
    -------------------------------------------------------------------------
DATA16_AN
  Relative segment, address: 0402 - 0403 (0x2 bytes), align: 0
  Segment part 14. ROOT       Intra module refs:   timer2_A0_init
           ENTRY                   ADDRESS         REF BY
           =====                   =======         ======
           TA2CCTL0                0402 
    -------------------------------------------------------------------------
DATA16_AN
  Relative segment, address: 0404 - 0405 (0x2 bytes), align: 0
  Segment part 15. ROOT       Intra module refs:   timer2_A0_init
           ENTRY                   ADDRESS         REF BY
           =====                   =======         ======
           TA2CCTL1                0404 
    -------------------------------------------------------------------------
DATA16_AN
  Relative segment, address: 0406 - 0407 (0x2 bytes), align: 0
  Segment part 16. ROOT       Intra module refs:   timer2_A0_init
           ENTRY                   ADDRESS         REF BY
           =====                   =======         ======
           TA2CCTL2                0406 
    -------------------------------------------------------------------------
DATA16_AN
  Relative segment, address: 0412 - 0413 (0x2 bytes), align: 0
  Segment part 17. ROOT       Intra module refs:   timer2_A0_init
           ENTRY                   ADDRESS         REF BY
           =====                   =======         ======
           TA2CCR0                 0412 
    -------------------------------------------------------------------------
DATA16_AN
  Relative segment, address: 0414 - 0415 (0x2 bytes), align: 0
  Segment part 18. ROOT       Intra module refs:   timer2_A0_init
           ENTRY                   ADDRESS         REF BY
           =====                   =======         ======
           TA2CCR1                 0414 
    -------------------------------------------------------------------------
DATA16_AN
  Relative segment, address: 0416 - 0417 (0x2 bytes), align: 0
  Segment part 19. ROOT       Intra module refs:   timer2_A0_init
           ENTRY                   ADDRESS         REF BY
           =====                   =======         ======
           TA2CCR2                 0416 
    -------------------------------------------------------------------------
DATA16_Z
  Relative segment, address: 2610 - 2610 (0x1 bytes), align: 0
  Segment part 24.            Intra module refs:   TIMER0_A0_ISR
           ENTRY                   ADDRESS         REF BY
           =====                   =======         ======
           timer_done_flag         2610 
    -------------------------------------------------------------------------
DATA16_I
  Relative segment, address: 2408 - 2409 (0x2 bytes), align: 1
  Segment part 25.            Intra module refs:   TIMER1_A0_ISR
           ENTRY                   ADDRESS         REF BY
           =====                   =======         ======
           timer_trigger_freq      2408            handleHostCommand (host_interface)
    -------------------------------------------------------------------------
DATA16_Z
  Relative segment, address: 2611 - 2611 (0x1 bytes), align: 0
  Segment part 27.            Intra module refs:   TIMER1_A0_ISR
           ENTRY                   ADDRESS         REF BY
           =====                   =======         ======
           next_trigger_time       2611            main (main)
    -------------------------------------------------------------------------
DATA16_Z
  Relative segment, address: 2612 - 2612 (0x1 bytes), align: 0
  Segment part 28.            Intra module refs:   tdc_trigger_measure
           ENTRY                   ADDRESS         REF BY
           =====                   =======         ======
           TDC720x_Measure_LT12ns
                                   2612            handleHostCommand (host_interface)
    -------------------------------------------------------------------------
DATA16_Z
  Relative segment, address: 2613 - 2613 (0x1 bytes), align: 0
  Segment part 29.
           ENTRY                   ADDRESS         REF BY
           =====                   =======         ======
           Measure_LT12ns_Method   2613            TDC720x_mode1_lt12ns (tdc720x_mode1_lt12ns)
                                                   USBCommunicationTask (main)
                                                   handleHostCommand (host_interface)
    -------------------------------------------------------------------------
DATA16_Z
  Relative segment, address: 2614 - 2614 (0x1 bytes), align: 0
  Segment part 30.            Intra module refs:   tdc_trigger_measure
           ENTRY                   ADDRESS         REF BY
           =====                   =======         ======
           TDC720x_Graph_Select    2614            handleHostCommand (host_interface)
    -------------------------------------------------------------------------
ISR_CODE
  Relative segment, address: 46EE - 46F3 (0x6 bytes), align: 1
  Segment part 40.            Intra module refs:   TIMER0_A0_ISR::??INTVEC 106
           ENTRY                   ADDRESS         REF BY
           =====                   =======         ======
           TIMER0_A0_ISR           46EE 
               interrupt function
               CSTACK = 00000000 ( 00000004 )
    -------------------------------------------------------------------------
<CODE> 1 (was CODE)
  Relative segment, address: 8EDC - 8EF9 (0x1e bytes), align: 1
  Segment part 36.
           ENTRY                   ADDRESS         REF BY
           =====                   =======         ======
           timer1_A0_init          8EDC            main (main)
               CSTACK = 00000000 ( 00000004 )
    -------------------------------------------------------------------------
<CODE> 1 (was CODE)
  Relative segment, address: 830E - 836F (0x62 bytes), align: 1
  Segment part 35.
           ENTRY                   ADDRESS         REF BY
           =====                   =======         ======
           timer2_A0_init          830E            main (main)
               CSTACK = 00000000 ( 00000006 )
    -------------------------------------------------------------------------
ISR_CODE
  Relative segment, address: 46F4 - 4701 (0xe bytes), align: 1
  Segment part 39.            Intra module refs:   TIMER2_A0_ISR::??INTVEC 88
           ENTRY                   ADDRESS         REF BY
           =====                   =======         ======
           TIMER2_A0_ISR           46F4 
               interrupt function
               CSTACK = 00000000 ( 00000004 )
    -------------------------------------------------------------------------
ISR_CODE
  Relative segment, address: 4702 - 471F (0x1e bytes), align: 1
  Segment part 38.            Intra module refs:   TIMER1_A0_ISR::??INTVEC 98
           ENTRY                   ADDRESS         REF BY
           =====                   =======         ======
           TIMER1_A0_ISR           4702 
               interrupt function
               CSTACK = 00000000 ( 00000006 )
    -------------------------------------------------------------------------
DATA16_Z
  Relative segment, address: 2615 - 2615 (0x1 bytes), align: 0
  Segment part 31.            Intra module refs:   TIMER1_A0_ISR
           LOCAL                   ADDRESS         
           =====                   =======         
           TIMER1_A0_ISR::delay_sec
                                   2615 
    -------------------------------------------------------------------------
<CODE> 1 (was CODE)
  Relative segment, address: 8CA0 - 8CCB (0x2c bytes), align: 1
  Segment part 34.
           ENTRY                   ADDRESS         REF BY
           =====                   =======         ======
           tdc_trigger_measure     8CA0            main (main)
               calls direct
               CSTACK = 00000000 ( 00000004 )
    -------------------------------------------------------------------------
<CODE> 1 (was CODE)
  Relative segment, address: 8C44 - 8C71 (0x2e bytes), align: 1
  Segment part 32.
           ENTRY                   ADDRESS         REF BY
           =====                   =======         ======
           wait_on_intb_pin        8C44            handle_TDC720x_plus_mux (tdc720x_mode1_lt12ns)
                                                   handle_two_TDC720x (tdc720x_mode1_lt12ns)
                                                   one_tdc_measure_results (tdc720x_measurement_control)
                                                   two_tdc_measure_results (tdc720x_measurement_control)
               CSTACK = 00000000 ( 00000004 )
    -------------------------------------------------------------------------
INTVEC
  Common segment, address: FF80 - FFD9 (0x5a bytes), align: 1
  Segment part 20. ROOT 
           ENTRY                   ADDRESS         REF BY
           =====                   =======         ======
           TIMER2_A0_ISR::??INTVEC 88
                                   FFD8 
    -------------------------------------------------------------------------
INTVEC
  Common segment, address: FF80 - FFE3 (0x64 bytes), align: 1
  Segment part 21. ROOT 
           ENTRY                   ADDRESS         REF BY
           =====                   =======         ======
           TIMER1_A0_ISR::??INTVEC 98
                                   FFE2 
    -------------------------------------------------------------------------
INTVEC
  Common segment, address: FF80 - FFEB (0x6c bytes), align: 1
  Segment part 22. ROOT 
           ENTRY                   ADDRESS         REF BY
           =====                   =======         ======
           TIMER0_A0_ISR::??INTVEC 106
                                   FFEA 
    -------------------------------------------------------------------------
DATA16_ID
  Relative segment, address: 468A - 468B (0x2 bytes), align: 1
  Segment part 26.            Intra module refs:   timer_trigger_freq

    *************************************************************************

  FILE NAME : C:\Users\a0415888\Documents\pwd\GIT_REPOS\TDC7200\tdc7200evm_fw\Debug\Obj\tlv.r43
  PROGRAM MODULE, NAME : tlv

  SEGMENTS IN THE MODULE
  ======================
<CODE> 1 (was CODE)
  Relative segment, address: 8690 - 86DF (0x50 bytes), align: 1
  Segment part 6.
           ENTRY                   ADDRESS         REF BY
           =====                   =======         ======
           TLV_getInfo             8690            USB_InitSerialStringDescriptor (usb)
               CSTACK = 00000000 ( 00000008 )

    *************************************************************************

  FILE NAME : C:\Users\a0415888\Documents\pwd\GIT_REPOS\TDC7200\tdc7200evm_fw\Debug\Obj\uart_commn.r43
  PROGRAM MODULE, NAME : uart_commn

  SEGMENTS IN THE MODULE
  ======================
DATA16_AN
  Relative segment, address: 0226 - 0227 (0x2 bytes), align: 0
  Segment part 2. ROOT        Intra module refs:   InitUART
           ENTRY                   ADDRESS         REF BY
           =====                   =======         ======
           _A_PBREN_L              0226 
           LOCAL                   ADDRESS         
           =====                   =======         
           PBREN                   0226 
           PBREN_H                 0227 
           PBREN_L                 0226 
    -------------------------------------------------------------------------
DATA16_AN
  Relative segment, address: 0600 - 0601 (0x2 bytes), align: 0
  Segment part 4. ROOT        Intra module refs:   InitUART
           ENTRY                   ADDRESS         REF BY
           =====                   =======         ======
           _A_UCA1CTLW0_L          0600 
           LOCAL                   ADDRESS         
           =====                   =======         
           UCA1CTLW0               0600 
           UCA1CTLW0_H             0601 
           UCA1CTLW0_L             0600 
    -------------------------------------------------------------------------
DATA16_AN
  Relative segment, address: 0606 - 0607 (0x2 bytes), align: 0
  Segment part 5. ROOT        Intra module refs:   InitUART
           ENTRY                   ADDRESS         REF BY
           =====                   =======         ======
           _A_UCA1BRW_L            0606 
           LOCAL                   ADDRESS         
           =====                   =======         
           UCA1BRW                 0606 
           UCA1BRW_H               0607 
           UCA1BRW_L               0606 
    -------------------------------------------------------------------------
DATA16_AN
  Relative segment, address: 0608 - 0608 (0x1 bytes), align: 0
  Segment part 6. ROOT        Intra module refs:   InitUART
           ENTRY                   ADDRESS         REF BY
           =====                   =======         ======
           UCA1MCTL                0608 
    -------------------------------------------------------------------------
DATA16_AN
  Relative segment, address: 060E - 060E (0x1 bytes), align: 0
  Segment part 7. ROOT        Intra module refs:   putsUART
           ENTRY                   ADDRESS         REF BY
           =====                   =======         ======
           UCA1TXBUF               060E 
    -------------------------------------------------------------------------
DATA16_AN
  Relative segment, address: 061C - 061D (0x2 bytes), align: 0
  Segment part 8. ROOT        Intra module refs:   InitUART
                                                   putsUART
           ENTRY                   ADDRESS         REF BY
           =====                   =======         ======
           _A_UCA1ICTL_L           061C 
           LOCAL                   ADDRESS         
           =====                   =======         
           UCA1ICTL                061C 
           UCA1ICTL_H              061D 
           UCA1ICTL_L              061C 
    -------------------------------------------------------------------------
<CODE> 1 (was CODE)
  Relative segment, address: 8A10 - 8A4B (0x3c bytes), align: 1
  Segment part 14.
           ENTRY                   ADDRESS         REF BY
           =====                   =======         ======
           InitUART                8A10            handleHostCommand (host_interface)
                                                   main (main)
               CSTACK = 00000000 ( 00000004 )
    -------------------------------------------------------------------------
<CODE> 1 (was CODE)
  Relative segment, address: 8C16 - 8C43 (0x2e bytes), align: 1
  Segment part 10.
           ENTRY                   ADDRESS         REF BY
           =====                   =======         ======
           putsUART                8C16            handleHostCommand (host_interface)
                                                   print_start2stopn (tdc720x_calculation)
               CSTACK = 00000000 ( 00000004 )

    *************************************************************************

  FILE NAME : C:\Users\a0415888\Documents\pwd\GIT_REPOS\TDC7200\tdc7200evm_fw\Debug\Obj\ucs.r43
  PROGRAM MODULE, NAME : ucs

  SEGMENTS IN THE MODULE
  ======================
<CODE> 1 (was CODE)
  Relative segment, address: 8892 - 88D3 (0x42 bytes), align: 1
  Segment part 18.
           ENTRY                   ADDRESS         REF BY
           =====                   =======         ======
           UCS_turnOnXT2WithTimeout
                                   8892            USB_enable (usb)
               CSTACK = 00000000 ( 00000004 )
    -------------------------------------------------------------------------
<CODE> 1 (was CODE)
  Relative segment, address: 92B4 - 92BB (0x8 bytes), align: 1
  Segment part 16.
           ENTRY                   ADDRESS         REF BY
           =====                   =======         ======
           UCS_turnOffXT2          92B4            USB_handleVbusOffEvent (usbEventHandling)
                                                   USB_suspend (usb)
               CSTACK = 00000000 ( 00000004 )

    *************************************************************************

  FILE NAME : C:\Users\a0415888\Documents\pwd\GIT_REPOS\TDC7200\tdc7200evm_fw\Debug\Obj\usb.r43
  PROGRAM MODULE, NAME : usb

  SEGMENTS IN THE MODULE
  ======================
DATA16_AN
  Relative segment, address: 0900 - 0901 (0x2 bytes), align: 0
  Segment part 1. ROOT        Intra module refs:   PWRVBUSoffHandler (UsbIsr)
                                                   PWRVBUSonHandler (UsbIsr)
                                                   USB_connect
                                                   USB_disable
                                                   USB_enable
                                                   USB_init
                                                   USB_reset
                                                   USB_suspend
           ENTRY                   ADDRESS         REF BY
           =====                   =======         ======
           _A_USBKEYID_L           0900 
           LOCAL                   ADDRESS         
           =====                   =======         
           USBKEYID                0900 
           USBKEYID_H              0901 
           USBKEYID_L              0900 
    -------------------------------------------------------------------------
DATA16_AN
  Relative segment, address: 0902 - 0903 (0x2 bytes), align: 0
  Segment part 2. ROOT        Intra module refs:   PWRVBUSoffHandler (UsbIsr)
                                                   USB_connect
                                                   USB_disable
                                                   USB_enable
                                                   USB_getConnectionInformation
                                                   USB_getConnectionState
           ENTRY                   ADDRESS         REF BY
           =====                   =======         ======
           _A_USBCNF_L             0902 
           LOCAL                   ADDRESS         
           =====                   =======         
           USBCNF                  0902 
           USBCNF_H                0903 
           USBCNF_L                0902 
    -------------------------------------------------------------------------
DATA16_AN
  Relative segment, address: 0904 - 0905 (0x2 bytes), align: 0
  Segment part 3. ROOT        Intra module refs:   USB_init
           ENTRY                   ADDRESS         REF BY
           =====                   =======         ======
           _A_USBPHYCTL_L          0904 
           LOCAL                   ADDRESS         
           =====                   =======         
           USBPHYCTL               0904 
           USBPHYCTL_H             0905 
           USBPHYCTL_L             0904 
    -------------------------------------------------------------------------
DATA16_AN
  Relative segment, address: 0908 - 0909 (0x2 bytes), align: 0
  Segment part 4. ROOT        Intra module refs:   PWRVBUSoffHandler (UsbIsr)
                                                   PWRVBUSonHandler (UsbIsr)
                                                   USB_connect
                                                   USB_enable
                                                   USB_getConnectionInformation
                                                   USB_getConnectionState
                                                   USB_init
           ENTRY                   ADDRESS         REF BY
           =====                   =======         ======
           _A_USBPWRCTL_L          0908 
           LOCAL                   ADDRESS         
           =====                   =======         
           USBPWRCTL               0908 
           USBPWRCTL_H             0909 
           USBPWRCTL_L             0908 
    -------------------------------------------------------------------------
DATA16_AN
  Relative segment, address: 0910 - 0911 (0x2 bytes), align: 0
  Segment part 5. ROOT        Intra module refs:   PWRVBUSoffHandler (UsbIsr)
                                                   USB_disable
                                                   USB_enable
                                                   USB_suspend
           ENTRY                   ADDRESS         REF BY
           =====                   =======         ======
           _A_USBPLLCTL_L          0910 
           LOCAL                   ADDRESS         
           =====                   =======         
           USBPLLCTL               0910 
           USBPLLCTL_H             0911 
           USBPLLCTL_L             0910 
    -------------------------------------------------------------------------
DATA16_AN
  Relative segment, address: 0912 - 0913 (0x2 bytes), align: 0
  Segment part 6. ROOT        Intra module refs:   USB_enable
           ENTRY                   ADDRESS         REF BY
           =====                   =======         ======
           _A_USBPLLDIVB_L         0912 
           LOCAL                   ADDRESS         
           =====                   =======         
           USBPLLDIVB              0912 
           USBPLLDIVB_H            0913 
           USBPLLDIVB_L            0912 
    -------------------------------------------------------------------------
DATA16_AN
  Relative segment, address: 0914 - 0915 (0x2 bytes), align: 0
  Segment part 7. ROOT        Intra module refs:   USB_enable
           ENTRY                   ADDRESS         REF BY
           =====                   =======         ======
           _A_USBPLLIR_L           0914 
           LOCAL                   ADDRESS         
           =====                   =======         
           USBPLLIR                0914 
           USBPLLIR_H              0915 
           USBPLLIR_L              0914 
    -------------------------------------------------------------------------
DATA16_AN
  Relative segment, address: 092E - 092E (0x1 bytes), align: 0
  Segment part 8. ROOT        Intra module refs:   USB_reset
                                                   usbDisableInEndpointInterrupt
                                                   usbRestoreInEndpointInterrupt
           ENTRY                   ADDRESS         REF BY
           =====                   =======         ======
           USBIEPIE                092E 
    -------------------------------------------------------------------------
DATA16_AN
  Relative segment, address: 092F - 092F (0x1 bytes), align: 0
  Segment part 9. ROOT        Intra module refs:   USB_reset
                                                   usbDisableOutEndpointInterrupt
                                                   usbRestoreOutEndpointInterrupt
           ENTRY                   ADDRESS         REF BY
           =====                   =======         ======
           USBOEPIE                092F 
    -------------------------------------------------------------------------
DATA16_AN
  Relative segment, address: 093C - 093C (0x1 bytes), align: 0
  Segment part 10. ROOT       Intra module refs:   IEP0InterruptHandler (UsbIsr)
                                                   OEP0InterruptHandler (UsbIsr)
                                                   SetupPacketInterruptHandler (UsbIsr)
                                                   USB_reset
                                                   USB_suspend
           ENTRY                   ADDRESS         REF BY
           =====                   =======         ======
           USBCTL                  093C 
    -------------------------------------------------------------------------
DATA16_AN
  Relative segment, address: 093D - 093D (0x1 bytes), align: 0
  Segment part 11. ROOT       Intra module refs:   USB_reset
                                                   USB_resume
                                                   USB_suspend
           ENTRY                   ADDRESS         REF BY
           =====                   =======         ======
           USBIE                   093D 
    -------------------------------------------------------------------------
DATA16_AN
  Relative segment, address: 093E - 093E (0x1 bytes), align: 0
  Segment part 12. ROOT       Intra module refs:   SetupPacketInterruptHandler (UsbIsr)
                                                   USB_reset
                                                   USB_resume
                                                   USB_suspend
                                                   iUsbInterruptHandler (UsbIsr)
                                                   usbDecodeAndProcessUsbRequest
                                                   usbInvalidRequest
           ENTRY                   ADDRESS         REF BY
           =====                   =======         ======
           USBIFG                  093E 
    -------------------------------------------------------------------------
DATA16_AN
  Relative segment, address: 093F - 093F (0x1 bytes), align: 0
  Segment part 13. ROOT       Intra module refs:   USB_reset
                                                   usbSetAddress
           ENTRY                   ADDRESS         REF BY
           =====                   =======         ======
           USBFUNADR               093F 
    -------------------------------------------------------------------------
DATA16_AN
  Relative segment, address: 016A - 016B (0x2 bytes), align: 0
  Segment part 17. ROOT       Intra module refs:   USB_determineFreq
           ENTRY                   ADDRESS         REF BY
           =====                   =======         ======
           _A_UCSCTL5_L            016A 
           LOCAL                   ADDRESS         
           =====                   =======         
           UCSCTL5                 016A 
           UCSCTL5_H               016B 
           UCSCTL5_L               016A 
    -------------------------------------------------------------------------
DATA16_Z
  Relative segment, address: 2616 - 2616 (0x1 bytes), align: 0
  Segment part 26.            Intra module refs:   USB_reset
                                                   usbGetConfiguration
                                                   usbSetConfiguration
           LOCAL                   ADDRESS         
           =====                   =======         
           bConfigurationNumber    2616 
    -------------------------------------------------------------------------
DATA16_Z
  Relative segment, address: 2617 - 2617 (0x1 bytes), align: 0
  Segment part 27.            Intra module refs:   USB_reset
                                                   usbGetInterface
                                                   usbGetInterfaceStatus
                                                   usbSetInterface
           LOCAL                   ADDRESS         
           =====                   =======         
           bInterfaceNumber        2617 
    -------------------------------------------------------------------------
DATA16_Z
  Relative segment, address: 246A - 246B (0x2 bytes), align: 1
  Segment part 28.            Intra module refs:   USB_reset
                                                   usbGetConfiguration
                                                   usbGetConfigurationDescriptor
                                                   usbGetDeviceDescriptor
                                                   usbGetDeviceStatus
                                                   usbGetEndpointStatus
                                                   usbGetInterface
                                                   usbGetInterfaceStatus
                                                   usbGetStringDescriptor
                                                   usbSendDataPacketOnEP0
                                                   usbSendNextPacketOnIEP0
                                                   usbSendZeroLengthPacketOnIEP0
           ENTRY                   ADDRESS         REF BY
           =====                   =======         ======
           wBytesRemainingOnIEP0   246A            usbGetLineCoding (UsbCdc)
    -------------------------------------------------------------------------
DATA16_Z
  Relative segment, address: 246C - 246D (0x2 bytes), align: 1
  Segment part 29.            Intra module refs:   USB_reset
                                                   usbReceiveDataPacketOnEP0
                                                   usbReceiveNextPacketOnOEP0
           ENTRY                   ADDRESS         REF BY
           =====                   =======         ======
           wBytesRemainingOnOEP0   246C 
    -------------------------------------------------------------------------
DATA16_Z
  Relative segment, address: 246E - 246F (0x2 bytes), align: 1
  Segment part 30.            Intra module refs:   usbSendDataPacketOnEP0
                                                   usbSendNextPacketOnIEP0
           LOCAL                   ADDRESS         
           =====                   =======         
           pbIEP0Buffer            246E 
    -------------------------------------------------------------------------
DATA16_Z
  Relative segment, address: 2470 - 2471 (0x2 bytes), align: 1
  Segment part 31.            Intra module refs:   usbReceiveDataPacketOnEP0
                                                   usbReceiveNextPacketOnOEP0
           LOCAL                   ADDRESS         
           =====                   =======         
           pbOEP0Buffer            2470 
    -------------------------------------------------------------------------
DATA16_Z
  Relative segment, address: 2618 - 2618 (0x1 bytes), align: 0
  Segment part 32.            Intra module refs:   usbSendDataPacketOnEP0
                                                   usbSendNextPacketOnIEP0
           LOCAL                   ADDRESS         
           =====                   =======         
           bHostAskMoreDataThanAvailable
                                   2618 
    -------------------------------------------------------------------------
DATA16_Z
  Relative segment, address: 2619 - 2620 (0x8 bytes), align: 0
  Segment part 33.            Intra module refs:   usbGetDeviceStatus
                                                   usbGetEndpointStatus
                                                   usbGetInterface
                                                   usbGetInterfaceStatus
           ENTRY                   ADDRESS         REF BY
           =====                   =======         ======
           abUsbRequestReturnData
                                   2619            SetupPacketInterruptHandler (UsbIsr)
                                                   usbGetLineCoding (UsbCdc)
    -------------------------------------------------------------------------
DATA16_Z
  Relative segment, address: 2621 - 2628 (0x8 bytes), align: 0
  Segment part 34.
           ENTRY                   ADDRESS         REF BY
           =====                   =======         ======
           abUsbRequestIncomingData
                                   2621            Handler_SetLineCoding (UsbCdc)
                                                   usbSetLineCoding (UsbCdc)
    -------------------------------------------------------------------------
DATA16_N
  Relative segment, address: 262D - 264E (0x22 bytes), align: 0
  Segment part 35.            Intra module refs:   USB_InitSerialStringDescriptor
                                                   usbGetStringDescriptor
           ENTRY                   ADDRESS         REF BY
           =====                   =======         ======
           abramSerialStringDescriptor
                                   262D 
    -------------------------------------------------------------------------
DATA16_Z
  Relative segment, address: 2629 - 2629 (0x1 bytes), align: 0
  Segment part 36.            Intra module refs:   USB_reset
                                                   usbReceiveDataPacketOnEP0
                                                   usbReceiveNextPacketOnOEP0
                                                   usbSendNextPacketOnIEP0
                                                   usbSendZeroLengthPacketOnIEP0
           ENTRY                   ADDRESS         REF BY
           =====                   =======         ======
           bStatusAction           2629            IEP0InterruptHandler (UsbIsr)
                                                   OEP0InterruptHandler (UsbIsr)
                                                   SetupPacketInterruptHandler (UsbIsr)
    -------------------------------------------------------------------------
DATA16_Z
  Relative segment, address: 262A - 262A (0x1 bytes), align: 0
  Segment part 37.            Intra module refs:   USB_disable
                                                   USB_enable
                                                   USB_getConnectionInformation
                                                   USB_getConnectionState
                                                   USB_reset
                                                   USB_resume
                                                   USB_suspend
           ENTRY                   ADDRESS         REF BY
           =====                   =======         ======
           bFunctionSuspended      262A            PWRVBUSoffHandler (UsbIsr)
                                                   USBCDC_getBytesInUSBBuffer (UsbCdc)
                                                   USBCDC_getInterfaceStatus (UsbCdc)
                                                   USBCDC_receiveData (UsbCdc)
                                                   USBCDC_sendData (UsbCdc)
    -------------------------------------------------------------------------
DATA16_Z
  Relative segment, address: 262B - 262B (0x1 bytes), align: 0
  Segment part 38.            Intra module refs:   USB_disable
                                                   USB_getConnectionInformation
                                                   USB_getConnectionState
                                                   USB_reset
                                                   usbSetConfiguration
           ENTRY                   ADDRESS         REF BY
           =====                   =======         ======
           bEnumerationStatus      262B            PWRVBUSoffHandler (UsbIsr)
                                                   USBCDC_getBytesInUSBBuffer (UsbCdc)
                                                   USBCDC_getInterfaceStatus (UsbCdc)
                                                   USBCDC_receiveData (UsbCdc)
                                                   USBCDC_sendData (UsbCdc)
    -------------------------------------------------------------------------
DATA16_Z
  Relative segment, address: 262C - 262C (0x1 bytes), align: 0
  Segment part 39.            Intra module refs:   USB_reset
                                                   usbClearDeviceFeature
                                                   usbGetDeviceStatus
                                                   usbSetDeviceFeature
           LOCAL                   ADDRESS         
           =====                   =======         
           bRemoteWakeup           262C 
    -------------------------------------------------------------------------
DATA16_Z
  Relative segment, address: 2472 - 2473 (0x2 bytes), align: 1
  Segment part 40.            Intra module refs:   USB_init
                                                   USB_setEnabledEvents
           ENTRY                   ADDRESS         REF BY
           =====                   =======         ======
           wUsbEventMask           2472            CdcToBufferFromHost (UsbCdc)
                                                   CdcToHostFromBuffer (UsbCdc)
                                                   USBCDC_receiveData (UsbCdc)
                                                   iUsbInterruptHandler (UsbIsr)
    -------------------------------------------------------------------------
DATA16_AN
  Relative segment, address: 2380 - 2387 (0x8 bytes), align: 0
  Segment part 18. ROOT       Intra module refs:   usbClearDeviceFeature
                                                   usbClearEndpointFeature
                                                   usbDecodeAndProcessUsbRequest
                                                   usbGetEndpointStatus
                                                   usbGetStringDescriptor
                                                   usbReceiveDataPacketOnEP0
                                                   usbSendDataPacketOnEP0
                                                   usbSetAddress
                                                   usbSetConfiguration
                                                   usbSetDeviceFeature
                                                   usbSetEndpointFeature
                                                   usbSetInterface
           ENTRY                   ADDRESS         REF BY
           =====                   =======         ======
           tSetupPacket            2380            Handler_SetLineCoding (UsbCdc)
                                                   OEP0InterruptHandler (UsbIsr)
                                                   SetupPacketInterruptHandler (UsbIsr)
                                                   usbGetLineCoding (UsbCdc)
                                                   usbSetControlLineState (UsbCdc)
    -------------------------------------------------------------------------
DATA16_AN
  Relative segment, address: 0920 - 0923 (0x4 bytes), align: 0
  Segment part 19. ROOT       Intra module refs:   USB_reset
                                                   usbClearOEP0ByteCount
                                                   usbGetEndpointStatus
                                                   usbReceiveNextPacketOnOEP0
                                                   usbSendNextPacketOnIEP0
                                                   usbSendZeroLengthPacketOnIEP0
                                                   usbStallEndpoint0
                                                   usbStallOEP0
           ENTRY                   ADDRESS         REF BY
           =====                   =======         ======
           tEndPoint0DescriptorBlock
                                   0920            IEP0InterruptHandler (UsbIsr)
                                                   OEP0InterruptHandler (UsbIsr)
                                                   iUsbInterruptHandler (UsbIsr)
    -------------------------------------------------------------------------
DATA16_AN
  Relative segment, address: 23C8 - 23FF (0x38 bytes), align: 0
  Segment part 20. ROOT       Intra module refs:   USB_reset
                                                   usbClearEndpointFeature
                                                   usbGetEndpointStatus
                                                   usbSetEndpointFeature
           ENTRY                   ADDRESS         REF BY
           =====                   =======         ======
           tInputEndPointDescriptorBlock
                                   23C8            CdcToHostFromBuffer (UsbCdc)
    -------------------------------------------------------------------------
DATA16_AN
  Relative segment, address: 2388 - 23BF (0x38 bytes), align: 0
  Segment part 21. ROOT       Intra module refs:   USB_reset
                                                   usbClearEndpointFeature
                                                   usbGetEndpointStatus
                                                   usbSetEndpointFeature
           ENTRY                   ADDRESS         REF BY
           =====                   =======         ======
           tOutputEndPointDescriptorBlock
                                   2388            CdcToBufferFromHost (UsbCdc)
                                                   USBCDC_getBytesInUSBBuffer (UsbCdc)
                                                   USBCDC_getInterfaceStatus (UsbCdc)
                                                   USBCDC_receiveData (UsbCdc)
    -------------------------------------------------------------------------
DATA16_AN
  Relative segment, address: 2378 - 237F (0x8 bytes), align: 0
  Segment part 22. ROOT       Intra module refs:   usbSendNextPacketOnIEP0
           ENTRY                   ADDRESS         REF BY
           =====                   =======         ======
           abIEP0Buffer            2378 
    -------------------------------------------------------------------------
DATA16_AN
  Relative segment, address: 2370 - 2377 (0x8 bytes), align: 0
  Segment part 23. ROOT       Intra module refs:   usbReceiveNextPacketOnOEP0
           ENTRY                   ADDRESS         REF BY
           =====                   =======         ======
           abOEP0Buffer            2370 
    -------------------------------------------------------------------------
DATA16_I
  Relative segment, address: 240A - 240B (0x2 bytes), align: 1
  Segment part 41.            Intra module refs:   USB_getVersion
           ENTRY                   ADDRESS         REF BY
           =====                   =======         ======
           VERSION                 240A 
    -------------------------------------------------------------------------
<CODE> 1 (was CODE)
  Relative segment, address: 92F8 - 92FD (0x6 bytes), align: 1
  Segment part 88.            Intra module refs:   USB_init
           ENTRY                   ADDRESS         REF BY
           =====                   =======         ======
           USB_getVersion          92F8 
               CSTACK = 00000000 ( 00000004 )
    -------------------------------------------------------------------------
<CODE> 1 (was CODE)
  Relative segment, address: 74D4 - 756B (0x98 bytes), align: 1
  Segment part 87.
           ENTRY                   ADDRESS         REF BY
           =====                   =======         ======
           USB_init                74D4            InitMCU (main)
               calls direct and indirect
               CSTACK = 00000000 ( 0000000C )
    -------------------------------------------------------------------------
<CODE> 1 (was CODE)
  Relative segment, address: 7204 - 72C9 (0xc6 bytes), align: 1
  Segment part 85.            Intra module refs:   USB_init
           ENTRY                   ADDRESS         REF BY
           =====                   =======         ======
           USB_InitSerialStringDescriptor
                                   7204 
               calls direct
               CSTACK = 00000000 ( 0000000A )
    -------------------------------------------------------------------------
<CODE> 1 (was CODE)
  Relative segment, address: 6C18 - 6D05 (0xee bytes), align: 1
  Segment part 84.            Intra module refs:   USB_resume
           ENTRY                   ADDRESS         REF BY
           =====                   =======         ======
           USB_enable              6C18            USB_handleVbusOnEvent (usbEventHandling)
               calls direct
               CSTACK = 00000000 ( 0000000C )
    -------------------------------------------------------------------------
<CODE> 1 (was CODE)
  Relative segment, address: 8E3E - 8E5F (0x22 bytes), align: 1
  Segment part 83.
           ENTRY                   ADDRESS         REF BY
           =====                   =======         ======
           USB_disable             8E3E            UNMI_ISR (main)
                                                   handleHostCommand (host_interface)
               CSTACK = 00000000 ( 00000004 )
    -------------------------------------------------------------------------
<CODE> 1 (was CODE)
  Relative segment, address: 92C4 - 92CB (0x8 bytes), align: 1
  Segment part 82.
           ENTRY                   ADDRESS         REF BY
           =====                   =======         ======
           USB_setEnabledEvents    92C4            InitMCU (main)
               CSTACK = 00000000 ( 00000004 )
    -------------------------------------------------------------------------
<CODE> 1 (was CODE)
  Relative segment, address: 62B6 - 643D (0x188 bytes), align: 1
  Segment part 80.
           ENTRY                   ADDRESS         REF BY
           =====                   =======         ======
           USB_reset               62B6            USB_handleVbusOnEvent (usbEventHandling)
                                                   iUsbInterruptHandler (UsbIsr)
               calls direct
               CSTACK = 00000000 ( 00000006 )
    -------------------------------------------------------------------------
<CODE> 1 (was CODE)
  Relative segment, address: 8F16 - 8F2F (0x1a bytes), align: 1
  Segment part 79.
           ENTRY                   ADDRESS         REF BY
           =====                   =======         ======
           USB_connect             8F16            USB_handleVbusOnEvent (usbEventHandling)
               CSTACK = 00000000 ( 00000004 )
    -------------------------------------------------------------------------
<CODE> 1 (was CODE)
  Relative segment, address: 8B8C - 8BB9 (0x2e bytes), align: 1
  Segment part 76.
           ENTRY                   ADDRESS         REF BY
           =====                   =======         ======
           USB_getConnectionInformation
                                   8B8C            InitMCU (main)
               CSTACK = 00000000 ( 00000004 )
    -------------------------------------------------------------------------
<CODE> 1 (was CODE)
  Relative segment, address: 769A - 772F (0x96 bytes), align: 1
  Segment part 75.
           ENTRY                   ADDRESS         REF BY
           =====                   =======         ======
           USB_getConnectionState
                                   769A            USBCommunicationTask (main)
               CSTACK = 00000000 ( 00000004 )
    -------------------------------------------------------------------------
<CODE> 1 (was CODE)
  Relative segment, address: 8B5C - 8B8B (0x30 bytes), align: 1
  Segment part 74.
           ENTRY                   ADDRESS         REF BY
           =====                   =======         ======
           USB_suspend             8B5C            iUsbInterruptHandler (UsbIsr)
               calls direct
               CSTACK = 00000000 ( 00000004 )
    -------------------------------------------------------------------------
<CODE> 1 (was CODE)
  Relative segment, address: 8F7A - 8F91 (0x18 bytes), align: 1
  Segment part 73.
           ENTRY                   ADDRESS         REF BY
           =====                   =======         ======
           USB_resume              8F7A            iUsbInterruptHandler (UsbIsr)
               calls direct
               CSTACK = 00000000 ( 00000004 )
    -------------------------------------------------------------------------
<CODE> 1 (was CODE)
  Relative segment, address: 92A0 - 92A9 (0xa bytes), align: 1
  Segment part 72.            Intra module refs:   usbClearDeviceFeature
                                                   usbGetStringDescriptor
                                                   usbInvalidRequest
                                                   usbSetAddress
                                                   usbSetDeviceFeature
                                                   usbSetEndpointFeature
           ENTRY                   ADDRESS         REF BY
           =====                   =======         ======
           usbStallEndpoint0       92A0 
               CSTACK = 00000000 ( 00000004 )
    -------------------------------------------------------------------------
<CODE> 1 (was CODE)
  Relative segment, address: 92DA - 92DF (0x6 bytes), align: 1
  Segment part 71.            Intra module refs:   usbGetConfiguration
                                                   usbGetConfigurationDescriptor
                                                   usbGetDeviceDescriptor
                                                   usbGetDeviceStatus
                                                   usbGetEndpointStatus
                                                   usbGetInterface
                                                   usbGetInterfaceStatus
                                                   usbGetStringDescriptor
                                                   usbReceiveDataPacketOnEP0
                                                   usbReceiveNextPacketOnOEP0
           ENTRY                   ADDRESS         REF BY
           =====                   =======         ======
           usbClearOEP0ByteCount   92DA 
               CSTACK = 00000000 ( 00000004 )
    -------------------------------------------------------------------------
<CODE> 1 (was CODE)
  Relative segment, address: 92E0 - 92E5 (0x6 bytes), align: 1
  Segment part 70.            Intra module refs:   usbReceiveNextPacketOnOEP0
                                                   usbSetAddress
                                                   usbSetConfiguration
                                                   usbSetInterface
           ENTRY                   ADDRESS         REF BY
           =====                   =======         ======
           usbStallOEP0            92E0 
               CSTACK = 00000000 ( 00000004 )
    -------------------------------------------------------------------------
<CODE> 1 (was CODE)
  Relative segment, address: 8094 - 8101 (0x6e bytes), align: 1
  Segment part 69.            Intra module refs:   usbSendDataPacketOnEP0
           ENTRY                   ADDRESS         REF BY
           =====                   =======         ======
           usbSendNextPacketOnIEP0
                                   8094            IEP0InterruptHandler (UsbIsr)
               CSTACK = 00000000 ( 00000004 )
    -------------------------------------------------------------------------
<CODE> 1 (was CODE)
  Relative segment, address: 8E80 - 8E9F (0x20 bytes), align: 1
  Segment part 68.            Intra module refs:   usbGetConfiguration
                                                   usbGetConfigurationDescriptor
                                                   usbGetDeviceDescriptor
                                                   usbGetDeviceStatus
                                                   usbGetEndpointStatus
                                                   usbGetInterface
                                                   usbGetInterfaceStatus
                                                   usbGetStringDescriptor
           ENTRY                   ADDRESS         REF BY
           =====                   =======         ======
           usbSendDataPacketOnEP0
                                   8E80            usbGetLineCoding (UsbCdc)
               calls direct
               CSTACK = 00000000 ( 00000004 )
    -------------------------------------------------------------------------
<CODE> 1 (was CODE)
  Relative segment, address: 859A - 85ED (0x54 bytes), align: 1
  Segment part 67.
           ENTRY                   ADDRESS         REF BY
           =====                   =======         ======
           usbReceiveNextPacketOnOEP0
                                   859A            OEP0InterruptHandler (UsbIsr)
               calls direct
               CSTACK = 00000000 ( 00000004 )
    -------------------------------------------------------------------------
<CODE> 1 (was CODE)
  Relative segment, address: 90B4 - 90C5 (0x12 bytes), align: 1
  Segment part 66.
           ENTRY                   ADDRESS         REF BY
           =====                   =======         ======
           usbReceiveDataPacketOnEP0
                                   90B4            usbSetLineCoding (UsbCdc)
               calls direct
               CSTACK = 00000000 ( 00000004 )
    -------------------------------------------------------------------------
<CODE> 1 (was CODE)
  Relative segment, address: 921C - 9229 (0xe bytes), align: 1
  Segment part 65.            Intra module refs:   usbClearDeviceFeature
                                                   usbClearEndpointFeature
                                                   usbSetAddress
                                                   usbSetConfiguration
                                                   usbSetDeviceFeature
                                                   usbSetEndpointFeature
                                                   usbSetInterface
           ENTRY                   ADDRESS         REF BY
           =====                   =======         ======
           usbSendZeroLengthPacketOnIEP0
                                   921C            usbSetControlLineState (UsbCdc)
               CSTACK = 00000000 ( 00000004 )
    -------------------------------------------------------------------------
<CODE> 1 (was CODE)
  Relative segment, address: 8996 - 89D3 (0x3e bytes), align: 1
  Segment part 64.
           ENTRY                   ADDRESS         REF BY
           =====                   =======         ======
           usbClearEndpointFeature
                                   8996            tUsbRequestList (descriptors)
               calls direct
               CSTACK = 00000000 ( 00000004 )
    -------------------------------------------------------------------------
<CODE> 1 (was CODE)
  Relative segment, address: 9068 - 907B (0x14 bytes), align: 1
  Segment part 63.
           ENTRY                   ADDRESS         REF BY
           =====                   =======         ======
           usbGetConfiguration     9068            tUsbRequestList (descriptors)
               calls direct
               CSTACK = 00000000 ( 00000004 )
    -------------------------------------------------------------------------
<CODE> 1 (was CODE)
  Relative segment, address: 8FEA - 8FFF (0x16 bytes), align: 1
  Segment part 62.
           ENTRY                   ADDRESS         REF BY
           =====                   =======         ======
           usbGetDeviceDescriptor
                                   8FEA            tUsbRequestList (descriptors)
               calls direct
               CSTACK = 00000000 ( 00000004 )
    -------------------------------------------------------------------------
<CODE> 1 (was CODE)
  Relative segment, address: 8FD4 - 8FE9 (0x16 bytes), align: 1
  Segment part 61.
           ENTRY                   ADDRESS         REF BY
           =====                   =======         ======
           usbGetConfigurationDescriptor
                                   8FD4            tUsbRequestList (descriptors)
               calls direct
               CSTACK = 00000000 ( 00000004 )
    -------------------------------------------------------------------------
<CODE> 1 (was CODE)
  Relative segment, address: 842E - 848B (0x5e bytes), align: 1
  Segment part 60.
           ENTRY                   ADDRESS         REF BY
           =====                   =======         ======
           usbGetStringDescriptor
                                   842E            tUsbRequestList (descriptors)
               calls direct
               CSTACK = 00000000 ( 00000006 )
    -------------------------------------------------------------------------
<CODE> 1 (was CODE)
  Relative segment, address: 8EA0 - 8EBD (0x1e bytes), align: 1
  Segment part 59.
           ENTRY                   ADDRESS         REF BY
           =====                   =======         ======
           usbGetInterface         8EA0            tUsbRequestList (descriptors)
               calls direct
               CSTACK = 00000000 ( 00000004 )
    -------------------------------------------------------------------------
<CODE> 1 (was CODE)
  Relative segment, address: 8D50 - 8D79 (0x2a bytes), align: 1
  Segment part 58.
           ENTRY                   ADDRESS         REF BY
           =====                   =======         ======
           usbGetDeviceStatus      8D50            tUsbRequestList (descriptors)
               calls direct
               CSTACK = 00000000 ( 00000004 )
    -------------------------------------------------------------------------
<CODE> 1 (was CODE)
  Relative segment, address: 8EBE - 8EDB (0x1e bytes), align: 1
  Segment part 57.
           ENTRY                   ADDRESS         REF BY
           =====                   =======         ======
           usbGetInterfaceStatus   8EBE            tUsbRequestList (descriptors)
               calls direct
               CSTACK = 00000000 ( 00000004 )
    -------------------------------------------------------------------------
<CODE> 1 (was CODE)
  Relative segment, address: 797A - 7A0B (0x92 bytes), align: 1
  Segment part 56.
           ENTRY                   ADDRESS         REF BY
           =====                   =======         ======
           usbGetEndpointStatus    797A            tUsbRequestList (descriptors)
               calls direct
               CSTACK = 00000000 ( 00000004 )
    -------------------------------------------------------------------------
<CODE> 1 (was CODE)
  Relative segment, address: 8E60 - 8E7F (0x20 bytes), align: 1
  Segment part 55.
           ENTRY                   ADDRESS         REF BY
           =====                   =======         ======
           usbSetAddress           8E60            tUsbRequestList (descriptors)
               calls direct
               CSTACK = 00000000 ( 00000004 )
    -------------------------------------------------------------------------
<CODE> 1 (was CODE)
  Relative segment, address: 8BBA - 8BE7 (0x2e bytes), align: 1
  Segment part 54.
           ENTRY                   ADDRESS         REF BY
           =====                   =======         ======
           usbSetConfiguration     8BBA            tUsbRequestList (descriptors)
               calls direct
               CSTACK = 00000000 ( 00000006 )
    -------------------------------------------------------------------------
<CODE> 1 (was CODE)
  Relative segment, address: 8F4A - 8F61 (0x18 bytes), align: 1
  Segment part 53.
           ENTRY                   ADDRESS         REF BY
           =====                   =======         ======
           usbClearDeviceFeature   8F4A            tUsbRequestList (descriptors)
               calls direct
               CSTACK = 00000000 ( 00000004 )
    -------------------------------------------------------------------------
<CODE> 1 (was CODE)
  Relative segment, address: 8F62 - 8F79 (0x18 bytes), align: 1
  Segment part 52.
           ENTRY                   ADDRESS         REF BY
           =====                   =======         ======
           usbSetDeviceFeature     8F62            tUsbRequestList (descriptors)
               calls direct
               CSTACK = 00000000 ( 00000004 )
    -------------------------------------------------------------------------
<CODE> 1 (was CODE)
  Relative segment, address: 880A - 884F (0x46 bytes), align: 1
  Segment part 51.
           ENTRY                   ADDRESS         REF BY
           =====                   =======         ======
           usbSetEndpointFeature   880A            tUsbRequestList (descriptors)
               calls direct
               CSTACK = 00000000 ( 00000004 )
    -------------------------------------------------------------------------
<CODE> 1 (was CODE)
  Relative segment, address: 910E - 911F (0x12 bytes), align: 1
  Segment part 50.
           ENTRY                   ADDRESS         REF BY
           =====                   =======         ======
           usbSetInterface         910E            tUsbRequestList (descriptors)
               calls direct
               CSTACK = 00000000 ( 00000004 )
    -------------------------------------------------------------------------
<CODE> 1 (was CODE)
  Relative segment, address: 91C8 - 91D5 (0xe bytes), align: 1
  Segment part 49.
           ENTRY                   ADDRESS         REF BY
           =====                   =======         ======
           usbInvalidRequest       91C8            tUsbRequestList (descriptors)
               calls direct
               CSTACK = 00000000 ( 00000004 )
    -------------------------------------------------------------------------
<CODE> 1 (was CODE)
  Relative segment, address: 77C4 - 7855 (0x92 bytes), align: 1
  Segment part 48.
           ENTRY                   ADDRESS         REF BY
           =====                   =======         ======
           usbDecodeAndProcessUsbRequest
                                   77C4            SetupPacketInterruptHandler (UsbIsr)
               calls indirect
               CSTACK = 00000000 ( 0000000C )
    -------------------------------------------------------------------------
<CODE> 1 (was CODE)
  Relative segment, address: 8BE8 - 8C15 (0x2e bytes), align: 1
  Segment part 47.
           ENTRY                   ADDRESS         REF BY
           =====                   =======         ======
           usbDisableInEndpointInterrupt
                                   8BE8            USBCDC_abortSend (UsbCdc)
                                                   USBCDC_getInterfaceStatus (UsbCdc)
                                                   USBCDC_sendData (UsbCdc)
               CSTACK = 00000000 ( 00000004 )
    -------------------------------------------------------------------------
<CODE> 1 (was CODE)
  Relative segment, address: 92F2 - 92F7 (0x6 bytes), align: 1
  Segment part 46.
           ENTRY                   ADDRESS         REF BY
           =====                   =======         ======
           usbRestoreInEndpointInterrupt
                                   92F2            USBCDC_abortSend (UsbCdc)
                                                   USBCDC_getInterfaceStatus (UsbCdc)
                                                   USBCDC_sendData (UsbCdc)
               CSTACK = 00000000 ( 00000004 )
    -------------------------------------------------------------------------
<CODE> 1 (was CODE)
  Relative segment, address: 8C72 - 8C9F (0x2e bytes), align: 1
  Segment part 45.
           ENTRY                   ADDRESS         REF BY
           =====                   =======         ======
           usbDisableOutEndpointInterrupt
                                   8C72            USBCDC_getBytesInUSBBuffer (UsbCdc)
                                                   USBCDC_getInterfaceStatus (UsbCdc)
                                                   USBCDC_receiveData (UsbCdc)
               CSTACK = 00000000 ( 00000004 )
    -------------------------------------------------------------------------
<CODE> 1 (was CODE)
  Relative segment, address: 92D4 - 92D9 (0x6 bytes), align: 1
  Segment part 44.
           ENTRY                   ADDRESS         REF BY
           =====                   =======         ======
           usbRestoreOutEndpointInterrupt
                                   92D4            USBCDC_getBytesInUSBBuffer (UsbCdc)
                                                   USBCDC_getInterfaceStatus (UsbCdc)
                                                   USBCDC_receiveData (UsbCdc)
               CSTACK = 00000000 ( 00000004 )
    -------------------------------------------------------------------------
<CODE> 1 (was CODE)
  Relative segment, address: 6876 - 69B1 (0x13c bytes), align: 1
  Segment part 43.            Intra module refs:   USB_enable
                                                   USB_init
           ENTRY                   ADDRESS         REF BY
           =====                   =======         ======
           USB_determineFreq       6876            PWRVBUSoffHandler (UsbIsr)
                                                   PWRVBUSonHandler (UsbIsr)
               CSTACK = 00000000 ( 00000008 )
    -------------------------------------------------------------------------
DATA16_ID
  Relative segment, address: 468C - 468D (0x2 bytes), align: 1
  Segment part 42.            Intra module refs:   VERSION
    -------------------------------------------------------------------------
DATA16_C
  Relative segment, address: 4649 - 4667 (0x1f bytes), align: 0
  Segment part 25.            Intra module refs:   Segment part 42

    *************************************************************************

  FILE NAME : C:\Users\a0415888\Documents\pwd\GIT_REPOS\TDC7200\tdc7200evm_fw\Debug\Obj\UsbCdc.r43
  PROGRAM MODULE, NAME : UsbCdc

  SEGMENTS IN THE MODULE
  ======================
DATA16_AN
  Relative segment, address: 0930 - 0930 (0x1 bytes), align: 0
  Segment part 1. ROOT        Intra module refs:   USBCDC_sendData
           ENTRY                   ADDRESS         REF BY
           =====                   =======         ======
           USBIEPIFG               0930 
    -------------------------------------------------------------------------
DATA16_Z
  Relative segment, address: 2474 - 247B (0x8 bytes), align: 1
  Segment part 3.             Intra module refs:   CdcResetData
                                                   Handler_SetLineCoding
                                                   usbGetLineCoding
           LOCAL                   ADDRESS         
           =====                   =======         
           CdcControl              2474 
    -------------------------------------------------------------------------
DATA16_Z
  Relative segment, address: 247C - 2485 (0xa bytes), align: 1
  Segment part 4.             Intra module refs:   CdcResetData
                                                   CdcToHostFromBuffer
                                                   USBCDC_abortSend
                                                   USBCDC_getInterfaceStatus
                                                   USBCDC_sendData
           LOCAL                   ADDRESS         
           =====                   =======         
           CdcWriteCtrl            247C 
    -------------------------------------------------------------------------
DATA16_Z
  Relative segment, address: 2486 - 2495 (0x10 bytes), align: 1
  Segment part 5.             Intra module refs:   CdcIsReceiveInProgress
                                                   CdcResetData
                                                   CdcToBufferFromHost
                                                   CopyUsbToBuff
                                                   USBCDC_getBytesInUSBBuffer
                                                   USBCDC_getInterfaceStatus
                                                   USBCDC_receiveData
           LOCAL                   ADDRESS         
           =====                   =======         
           CdcReadCtrl             2486 
    -------------------------------------------------------------------------
<CODE> 1 (was CODE)
  Relative segment, address: 89D4 - 8A0F (0x3c bytes), align: 1
  Segment part 21.
           ENTRY                   ADDRESS         REF BY
           =====                   =======         ======
           CdcResetData            89D4            USB_reset (usb)
               calls direct
               CSTACK = 00000000 ( 00000004 )
    -------------------------------------------------------------------------
<CODE> 1 (was CODE)
  Relative segment, address: 7730 - 77C3 (0x94 bytes), align: 1
  Segment part 20.
           ENTRY                   ADDRESS         REF BY
           =====                   =======         ======
           USBCDC_sendData         7730            USBCDC_sendDataInBackground (usbConstructs)
               calls direct
               CSTACK = 00000000 ( 0000000C )
    -------------------------------------------------------------------------
<CODE> 1 (was CODE)
  Relative segment, address: 5EA6 - 6101 (0x25c bytes), align: 1
  Segment part 19.
           ENTRY                   ADDRESS         REF BY
           =====                   =======         ======
           CdcToHostFromBuffer     5EA6            iUsbInterruptHandler (UsbIsr)
               calls direct and indirect
               CSTACK = 00000000 ( 00000010 )
    -------------------------------------------------------------------------
<CODE> 1 (was CODE)
  Relative segment, address: 8542 - 8599 (0x58 bytes), align: 1
  Segment part 18.
           ENTRY                   ADDRESS         REF BY
           =====                   =======         ======
           USBCDC_abortSend        8542            USBCommunicationTask (main)
               calls direct
               CSTACK = 00000000 ( 00000008 )
    -------------------------------------------------------------------------
<CODE> 1 (was CODE)
  Relative segment, address: 7604 - 7699 (0x96 bytes), align: 1
  Segment part 17.            Intra module refs:   CdcToBufferFromHost
                                                   USBCDC_receiveData
           ENTRY                   ADDRESS         REF BY
           =====                   =======         ======
           CopyUsbToBuff           7604 
               calls indirect
               CSTACK = 00000000 ( 0000000C )
    -------------------------------------------------------------------------
<CODE> 1 (was CODE)
  Relative segment, address: 5714 - 59D7 (0x2c4 bytes), align: 1
  Segment part 16.
           ENTRY                   ADDRESS         REF BY
           =====                   =======         ======
           USBCDC_receiveData      5714            USBCDC_receiveDataInBuffer (usbConstructs)
               calls direct
               CSTACK = 00000000 ( 00000010 )
    -------------------------------------------------------------------------
<CODE> 1 (was CODE)
  Relative segment, address: 65AC - 6713 (0x168 bytes), align: 1
  Segment part 15.
           ENTRY                   ADDRESS         REF BY
           =====                   =======         ======
           CdcToBufferFromHost     65AC            iUsbInterruptHandler (UsbIsr)
               calls direct
               CSTACK = 00000000 ( 0000000C )
    -------------------------------------------------------------------------
<CODE> 1 (was CODE)
  Relative segment, address: 9054 - 9067 (0x14 bytes), align: 1
  Segment part 14.
           ENTRY                   ADDRESS         REF BY
           =====                   =======         ======
           CdcIsReceiveInProgress
                                   9054            iUsbInterruptHandler (UsbIsr)
               CSTACK = 00000000 ( 00000004 )
    -------------------------------------------------------------------------
<CODE> 1 (was CODE)
  Relative segment, address: 713E - 7203 (0xc6 bytes), align: 1
  Segment part 11.
           ENTRY                   ADDRESS         REF BY
           =====                   =======         ======
           USBCDC_getInterfaceStatus
                                   713E            USBCDC_sendDataInBackground (usbConstructs)
                                                   USBCommunicationTask (main)
               calls direct
               CSTACK = 00000000 ( 00000014 )
    -------------------------------------------------------------------------
<CODE> 1 (was CODE)
  Relative segment, address: 78E8 - 7979 (0x92 bytes), align: 1
  Segment part 10.
           ENTRY                   ADDRESS         REF BY
           =====                   =======         ======
           USBCDC_getBytesInUSBBuffer
                                   78E8            USBCDC_receiveDataInBuffer (usbConstructs)
                                                   iUsbInterruptHandler (UsbIsr)
               calls direct
               CSTACK = 00000000 ( 0000000C )
    -------------------------------------------------------------------------
<CODE> 1 (was CODE)
  Relative segment, address: 7EB6 - 7F31 (0x7c bytes), align: 1
  Segment part 9.
           ENTRY                   ADDRESS         REF BY
           =====                   =======         ======
           usbGetLineCoding        7EB6            tUsbRequestList (descriptors)
               calls direct
               CSTACK = 00000000 ( 00000004 )
    -------------------------------------------------------------------------
<CODE> 1 (was CODE)
  Relative segment, address: 9238 - 9243 (0xc bytes), align: 1
  Segment part 8.
           ENTRY                   ADDRESS         REF BY
           =====                   =======         ======
           usbSetLineCoding        9238            tUsbRequestList (descriptors)
               calls direct
               CSTACK = 00000000 ( 00000004 )
    -------------------------------------------------------------------------
<CODE> 1 (was CODE)
  Relative segment, address: 902C - 903F (0x14 bytes), align: 1
  Segment part 7.
           ENTRY                   ADDRESS         REF BY
           =====                   =======         ======
           usbSetControlLineState
                                   902C            tUsbRequestList (descriptors)
               calls direct
               CSTACK = 00000000 ( 00000004 )
    -------------------------------------------------------------------------
<CODE> 1 (was CODE)
  Relative segment, address: 7A9C - 7B29 (0x8e bytes), align: 1
  Segment part 6.
           ENTRY                   ADDRESS         REF BY
           =====                   =======         ======
           Handler_SetLineCoding   7A9C            OEP0InterruptHandler (UsbIsr)
               calls direct
               CSTACK = 00000000 ( 0000000E )

    *************************************************************************

  FILE NAME : C:\Users\a0415888\Documents\pwd\GIT_REPOS\TDC7200\tdc7200evm_fw\Debug\Obj\usbConstructs.r43
  PROGRAM MODULE, NAME : usbConstructs

  SEGMENTS IN THE MODULE
  ======================
<CODE> 1 (was CODE)
  Relative segment, address: 816E - 81D9 (0x6c bytes), align: 1
  Segment part 3.
           ENTRY                   ADDRESS         REF BY
           =====                   =======         ======
           USBCDC_sendDataInBackground
                                   816E            USBCommunicationTask (main)
               calls direct
               CSTACK = 00000000 ( 00000018 )
    -------------------------------------------------------------------------
<CODE> 1 (was CODE)
  Relative segment, address: 8640 - 868F (0x50 bytes), align: 1
  Segment part 2.
           ENTRY                   ADDRESS         REF BY
           =====                   =======         ======
           USBCDC_receiveDataInBuffer
                                   8640            USBCommunicationTask (main)
               calls direct
               CSTACK = 00000000 ( 00000010 )

    *************************************************************************

  FILE NAME : C:\Users\a0415888\Documents\pwd\GIT_REPOS\TDC7200\tdc7200evm_fw\Debug\Obj\usbdma.r43
  PROGRAM MODULE, NAME : usbdma

  SEGMENTS IN THE MODULE
  ======================
DATA16_Z
  Relative segment, address: 2496 - 2499 (0x4 bytes), align: 1
  Segment part 3.             Intra module refs:   USB_initMemcpy
           ENTRY                   ADDRESS         REF BY
           =====                   =======         ======
           USB_TX_memcpy           2496            CdcToHostFromBuffer (UsbCdc)
    -------------------------------------------------------------------------
DATA16_Z
  Relative segment, address: 249A - 249D (0x4 bytes), align: 1
  Segment part 4.             Intra module refs:   USB_initMemcpy
           ENTRY                   ADDRESS         REF BY
           =====                   =======         ======
           USB_RX_memcpy           249A            CopyUsbToBuff (UsbCdc)
    -------------------------------------------------------------------------
<CODE> 1 (was CODE)
  Relative segment, address: 8E1A - 8E3D (0x24 bytes), align: 1
  Segment part 7.             Intra module refs:   USB_initMemcpy
           ENTRY                   ADDRESS         REF BY
           =====                   =======         ======
           memcpyV                 8E1A 
               CSTACK = 00000000 ( 00000008 )
    -------------------------------------------------------------------------
<CODE> 1 (was CODE)
  Relative segment, address: 848C - 84E9 (0x5e bytes), align: 1
  Segment part 6.             Intra module refs:   USB_initMemcpy
           ENTRY                   ADDRESS         REF BY
           =====                   =======         ======
           memcpyDMA               848C 
               calls direct
               CSTACK = 00000000 ( 0000000C )
    -------------------------------------------------------------------------
<CODE> 1 (was CODE)
  Relative segment, address: 81DA - 8241 (0x68 bytes), align: 1
  Segment part 5.
           ENTRY                   ADDRESS         REF BY
           =====                   =======         ======
           USB_initMemcpy          81DA            USB_init (usb)
               calls direct
               CSTACK = 00000000 ( 0000000E )

    *************************************************************************

  FILE NAME : C:\Users\a0415888\Documents\pwd\GIT_REPOS\TDC7200\tdc7200evm_fw\Debug\Obj\usbEventHandling.r43
  PROGRAM MODULE, NAME : usbEventHandling

  SEGMENTS IN THE MODULE
  ======================
<CODE> 1 (was CODE)
  Relative segment, address: 9332 - 9335 (0x4 bytes), align: 1
  Segment part 13.
           ENTRY                   ADDRESS         REF BY
           =====                   =======         ======
           USB_handleClockEvent    9332            iUsbInterruptHandler (UsbIsr)
               CSTACK = 00000000 ( 00000004 )
    -------------------------------------------------------------------------
<CODE> 1 (was CODE)
  Relative segment, address: 9040 - 9053 (0x14 bytes), align: 1
  Segment part 12.
           ENTRY                   ADDRESS         REF BY
           =====                   =======         ======
           USB_handleVbusOnEvent   9040            InitMCU (main)
                                                   iUsbInterruptHandler (UsbIsr)
               calls direct
               CSTACK = 00000000 ( 00000004 )
    -------------------------------------------------------------------------
<CODE> 1 (was CODE)
  Relative segment, address: 92CC - 92D3 (0x8 bytes), align: 1
  Segment part 11.
           ENTRY                   ADDRESS         REF BY
           =====                   =======         ======
           USB_handleVbusOffEvent
                                   92CC            iUsbInterruptHandler (UsbIsr)
               calls direct
               CSTACK = 00000000 ( 00000004 )
    -------------------------------------------------------------------------
<CODE> 1 (was CODE)
  Relative segment, address: 931A - 931D (0x4 bytes), align: 1
  Segment part 10.
           ENTRY                   ADDRESS         REF BY
           =====                   =======         ======
           USB_handleResetEvent    931A            iUsbInterruptHandler (UsbIsr)
               CSTACK = 00000000 ( 00000004 )
    -------------------------------------------------------------------------
<CODE> 1 (was CODE)
  Relative segment, address: 930A - 930D (0x4 bytes), align: 1
  Segment part 9.
           ENTRY                   ADDRESS         REF BY
           =====                   =======         ======
           USB_handleSuspendEvent
                                   930A            iUsbInterruptHandler (UsbIsr)
               CSTACK = 00000000 ( 00000004 )
    -------------------------------------------------------------------------
<CODE> 1 (was CODE)
  Relative segment, address: 9306 - 9309 (0x4 bytes), align: 1
  Segment part 8.
           ENTRY                   ADDRESS         REF BY
           =====                   =======         ======
           USB_handleResumeEvent   9306            iUsbInterruptHandler (UsbIsr)
               CSTACK = 00000000 ( 00000004 )
    -------------------------------------------------------------------------
<CODE> 1 (was CODE)
  Relative segment, address: 9326 - 9329 (0x4 bytes), align: 1
  Segment part 7.
           ENTRY                   ADDRESS         REF BY
           =====                   =======         ======
           USB_handleEnumerationCompleteEvent
                                   9326            usbSetConfiguration (usb)
               CSTACK = 00000000 ( 00000004 )
    -------------------------------------------------------------------------
<CODE> 1 (was CODE)
  Relative segment, address: 92BC - 92C3 (0x8 bytes), align: 1
  Segment part 6.
           ENTRY                   ADDRESS         REF BY
           =====                   =======         ======
           USBCDC_handleDataReceived
                                   92BC            CdcToBufferFromHost (UsbCdc)
                                                   iUsbInterruptHandler (UsbIsr)
               CSTACK = 00000000 ( 00000004 )
    -------------------------------------------------------------------------
<CODE> 1 (was CODE)
  Relative segment, address: 9312 - 9315 (0x4 bytes), align: 1
  Segment part 5.
           ENTRY                   ADDRESS         REF BY
           =====                   =======         ======
           USBCDC_handleSendCompleted
                                   9312            CdcToHostFromBuffer (UsbCdc)
               CSTACK = 00000000 ( 00000004 )
    -------------------------------------------------------------------------
<CODE> 1 (was CODE)
  Relative segment, address: 932E - 9331 (0x4 bytes), align: 1
  Segment part 4.
           ENTRY                   ADDRESS         REF BY
           =====                   =======         ======
           USBCDC_handleReceiveCompleted
                                   932E            CdcToBufferFromHost (UsbCdc)
                                                   USBCDC_receiveData (UsbCdc)
               CSTACK = 00000000 ( 00000004 )
    -------------------------------------------------------------------------
<CODE> 1 (was CODE)
  Relative segment, address: 931E - 9321 (0x4 bytes), align: 1
  Segment part 3.
           ENTRY                   ADDRESS         REF BY
           =====                   =======         ======
           USBCDC_handleSetLineCoding
                                   931E            Handler_SetLineCoding (UsbCdc)
               CSTACK = 00000000 ( 00000004 )
    -------------------------------------------------------------------------
<CODE> 1 (was CODE)
  Relative segment, address: 930E - 9311 (0x4 bytes), align: 1
  Segment part 2.
           ENTRY                   ADDRESS         REF BY
           =====                   =======         ======
           USBCDC_handleSetControlLineState
                                   930E            usbSetControlLineState (UsbCdc)
               CSTACK = 00000000 ( 00000004 )

    *************************************************************************

  FILE NAME : C:\Users\a0415888\Documents\pwd\GIT_REPOS\TDC7200\tdc7200evm_fw\Debug\Obj\UsbIsr.r43
  PROGRAM MODULE, NAME : UsbIsr

  SEGMENTS IN THE MODULE
  ======================
DATA16_AN
  Relative segment, address: 0932 - 0933 (0x2 bytes), align: 0
  Segment part 5. ROOT        Intra module refs:   iUsbInterruptHandler
           ENTRY                   ADDRESS         REF BY
           =====                   =======         ======
           _A_USBVECINT_L          0932 
           LOCAL                   ADDRESS         
           =====                   =======         
           USBVECINT               0932 
           USBVECINT_H             0933 
           USBVECINT_L             0932 
    -------------------------------------------------------------------------
ISR_CODE
  Relative segment, address: 4720 - 4861 (0x142 bytes), align: 1
  Segment part 15.            Intra module refs:   iUsbInterruptHandler::??INTVEC 102
           ENTRY                   ADDRESS         REF BY
           =====                   =======         ======
           iUsbInterruptHandler    4720 
               interrupt function
               calls direct
               CSTACK = 00000000 ( 00000010 )
    -------------------------------------------------------------------------
<CODE> 1 (was CODE)
  Relative segment, address: 8916 - 8955 (0x40 bytes), align: 1
  Segment part 14.            Intra module refs:   iUsbInterruptHandler
           ENTRY                   ADDRESS         REF BY
           =====                   =======         ======
           SetupPacketInterruptHandler
                                   8916 
               calls direct
               CSTACK = 00000000 ( 00000004 )
    -------------------------------------------------------------------------
<CODE> 1 (was CODE)
  Relative segment, address: 7F32 - 7FA9 (0x78 bytes), align: 1
  Segment part 13.            Intra module refs:   iUsbInterruptHandler
           ENTRY                   ADDRESS         REF BY
           =====                   =======         ======
           PWRVBUSoffHandler       7F32 
               calls direct
               CSTACK = 00000000 ( 00000008 )
    -------------------------------------------------------------------------
<CODE> 1 (was CODE)
  Relative segment, address: 8102 - 816D (0x6c bytes), align: 1
  Segment part 12.            Intra module refs:   iUsbInterruptHandler
           ENTRY                   ADDRESS         REF BY
           =====                   =======         ======
           PWRVBUSonHandler        8102 
               calls direct
               CSTACK = 00000000 ( 00000008 )
    -------------------------------------------------------------------------
<CODE> 1 (was CODE)
  Relative segment, address: 8F30 - 8F49 (0x1a bytes), align: 1
  Segment part 11.            Intra module refs:   iUsbInterruptHandler
           ENTRY                   ADDRESS         REF BY
           =====                   =======         ======
           IEP0InterruptHandler    8F30 
               calls direct
               CSTACK = 00000000 ( 00000004 )
    -------------------------------------------------------------------------
<CODE> 1 (was CODE)
  Relative segment, address: 8A4C - 8A83 (0x38 bytes), align: 1
  Segment part 10.            Intra module refs:   iUsbInterruptHandler
           ENTRY                   ADDRESS         REF BY
           =====                   =======         ======
           OEP0InterruptHandler    8A4C 
               calls direct
               CSTACK = 00000000 ( 00000006 )
    -------------------------------------------------------------------------
INTVEC
  Common segment, address: FF80 - FFE7 (0x68 bytes), align: 1
  Segment part 8. ROOT 
           ENTRY                   ADDRESS         REF BY
           =====                   =======         ======
           iUsbInterruptHandler::??INTVEC 102
                                   FFE6 

    *************************************************************************

  FILE NAME : C:\Users\a0415888\Documents\pwd\GIT_REPOS\TDC7200\tdc7200evm_fw\Debug\Obj\usci_a_spi.r43
    *************************************************************************

  FILE NAME : C:\Users\a0415888\Documents\pwd\GIT_REPOS\TDC7200\tdc7200evm_fw\Debug\Obj\usci_a_uart.r43
    *************************************************************************

  FILE NAME : C:\Users\a0415888\Documents\pwd\GIT_REPOS\TDC7200\tdc7200evm_fw\Debug\Obj\usci_b_i2c.r43
    *************************************************************************

  FILE NAME : C:\Users\a0415888\Documents\pwd\GIT_REPOS\TDC7200\tdc7200evm_fw\Debug\Obj\usci_b_spi.r43
    *************************************************************************

  FILE NAME : C:\Users\a0415888\Documents\pwd\GIT_REPOS\TDC7200\tdc7200evm_fw\Debug\Obj\wdt_a.r43
    *************************************************************************

  FILE NAME : C:\Program Files (x86)\IAR Systems\Embedded Workbench 7.0\430\lib\dlib\dl430xlsfn.r43
  LIBRARY MODULE, NAME : ?__dbg_break

  SEGMENTS IN THE MODULE
  ======================
<CODE> 1 (was CODE)
  Relative segment, address: 9336 - 9337 (0x2 bytes), align: 1
  Segment part 2.
           ENTRY                   ADDRESS         REF BY
           =====                   =======         ======
           __DebugBreak            9336            __exit (?__exit)

    -------------------------------------------------------------------------
  LIBRARY MODULE, NAME : ?__exit

  SEGMENTS IN THE MODULE
  ======================
<CODE> 1 (was CODE)
  Relative segment, address: 8FA8 - 8FBD (0x16 bytes), align: 1
  Segment part 2.
           ENTRY                   ADDRESS         REF BY
           =====                   =======         ======
           __exit                  8FA8            Segment part 6 (?_exit)
                                                   _exit (?_exit)
               calls direct

    -------------------------------------------------------------------------
  LIBRARY MODULE, NAME : ?_exit

  SEGMENTS IN THE MODULE
  ======================
<CODE> 1 (was CODE)
  Relative segment, address: 9302, align: 1
  Segment part 0.
           ENTRY                   ADDRESS         REF BY
           =====                   =======         ======
           _exit                   9302            exit (?exit)
    -------------------------------------------------------------------------
<CODE> 1 (was CODE)
  Relative segment, address: 9302 - 9305 (0x4 bytes), align: 1
  Segment part 6.             Intra module refs:   _exit

    -------------------------------------------------------------------------
  LIBRARY MODULE, NAME : ?cstart

  SEGMENTS IN THE MODULE
  ======================
CSTACK
  Relative segment, address: 4360, align: 1
  Segment part 1.
    -------------------------------------------------------------------------
DATA16_Z
  Relative segment, address: 249E, align: 1
  Segment part 2.
    -------------------------------------------------------------------------
DATA16_I
  Relative segment, address: 240C, align: 1
  Segment part 3.
    -------------------------------------------------------------------------
DATA16_ID
  Relative segment, address: 468E, align: 1
  Segment part 4.
    -------------------------------------------------------------------------
CODE_I
  Relative segment, address: 2650, align: 1
  Segment part 5.
    -------------------------------------------------------------------------
CODE_ID
  Relative segment, address: 933A, align: 1
  Segment part 6.
    -------------------------------------------------------------------------
DATA20_Z
  Relative segment, address: 2650, align: 1
  Segment part 7.
    -------------------------------------------------------------------------
DATA20_I
  Relative segment, address: 2650, align: 1
  Segment part 8.
    -------------------------------------------------------------------------
DATA20_ID
  Relative segment, address: 933A, align: 1
  Segment part 9.
    -------------------------------------------------------------------------
DATA20_C
  Relative segment, address: 933A, align: 1
  Segment part 10.
    -------------------------------------------------------------------------
DATA20_HEAP
  Relative segment, address: 2650, align: 1
  Segment part 11.
    -------------------------------------------------------------------------
DATA20_N
  Relative segment, address: 2650, align: 1
  Segment part 12.
    -------------------------------------------------------------------------
CSTART
  Relative segment, address: 4690 - 4693 (0x4 bytes), align: 1
  Segment part 15.
           ENTRY                   ADDRESS         REF BY
           =====                   =======         ======
           __program_start         4690            ?reset_vector (?reset_vector)
                                                   Absolute parts (?ABS_ENTRY_MOD)
           ?cstart_begin           4690 
    -------------------------------------------------------------------------
CSTART
  Relative segment, address: 4694 - 469F (0xc bytes), align: 1
  Segment part 19.
           ENTRY                   ADDRESS         REF BY
           =====                   =======         ======
           ?cstart_init_zero       4694            CdcControl (UsbCdc)
                                                   CdcReadCtrl (UsbCdc)
                                                   CdcWriteCtrl (UsbCdc)
                                                   Measure_LT12ns_Method (timer_queue)
                                                   TDC720x_Graph_Select (timer_queue)
                                                   TDC720x_Measure_LT12ns (timer_queue)
                                                   TDC720x_PQBufferReady (main)
                                                   TDC720x_Parallel_Read (tdc720x_measurement_control)
                                                   TDC720x_UART_Stream (host_interface)
                                                   TDC720x_XYBufferReady (main)
                                                   TDC720x_address (host_interface)
                                                   TIMER1_A0_ISR::delay_sec (timer_queue)
                                                   USB_RX_memcpy (usbdma)
                                                   USB_TX_memcpy (usbdma)
                                                   abUsbRequestIncomingData (usb)
                                                   abUsbRequestReturnData (usb)
                                                   all_data (host_interface)
                                                   bCDCDataReceived_event (main)
                                                   bConfigurationNumber (usb)
                                                   bEnumerationStatus (usb)
                                                   bFunctionSuspended (usb)
                                                   bHostAskMoreDataThanAvailable (usb)
                                                   bInterfaceNumber (usb)
                                                   bRemoteWakeup (usb)
                                                   bStatusAction (usb)
                                                   bufferP (main)
                                                   bufferQ (main)
                                                   bufferX (main)
                                                   bufferY (main)
                                                   ccnt (tdc720x_calculation)
                                                   cmdResponseString (main)
                                                   current_tdc (main)
                                                   double_resolution (main)
                                                   err_count (main)
                                                   graph_delay_sweep_state (main)
                                                   meas_result_regrs (tdc720x_calculation)
                                                   next_trigger_time (timer_queue)
                                                   norm_lsb (tdc720x_calculation)
                                                   outString (tdc720x_calculation)
                                                   pbIEP0Buffer (usb)
                                                   pbOEP0Buffer (usb)
                                                   save1_tdc7200_mode (host_interface)
                                                   save2_tdc7200_mode (host_interface)
                                                   save_default_timer_period (host_interface)
                                                   save_mode (host_interface)
                                                   save_timer_trig_freq (host_interface)
                                                   single_shot_measure_state (main)
                                                   start2stop (tdc720x_calculation)
                                                   timer_done_flag (timer_queue)
                                                   tof_graph_state (main)
                                                   ubuf (main)
                                                   vbuf (main)
                                                   w (main)
                                                   wBytesRemainingOnIEP0 (usb)
                                                   wBytesRemainingOnOEP0 (usb)
                                                   wUsbEventMask (usb)
    -------------------------------------------------------------------------
CSTART
  Relative segment, address: 46A0 - 46AF (0x10 bytes), align: 1
  Segment part 20.
           ENTRY                   ADDRESS         REF BY
           =====                   =======         ======
           ?cstart_init_copy       46A0            TDC720xEVM_Device (main)
                                                   VERSION (usb)
                                                   mbuf (main)
                                                   nbuf (main)
                                                   tdc_clk_period (tdc720x_calculation)
                                                   timer_trigger_freq (timer_queue)
    -------------------------------------------------------------------------
CSTART
  Relative segment, address: 46B0 - 46B7 (0x8 bytes), align: 1
  Segment part 26.            Intra module refs:   Segment part 15
           ENTRY                   ADDRESS         REF BY
           =====                   =======         ======
           ?cstart_call_main       46B0 
           ?cstart_end             46B8 
    -------------------------------------------------------------------------
CODE_ID
  Relative segment, address: 933A, align: 1
  Segment part 27.            Intra module refs:   Segment part 5

    -------------------------------------------------------------------------
  LIBRARY MODULE, NAME : ?reset_vector

  SEGMENTS IN THE MODULE
  ======================
RESET
  Relative segment, address: FFFE - FFFF (0x2 bytes), align: 1
  Segment part 0.
           ENTRY                   ADDRESS         REF BY
           =====                   =======         ======
           ?reset_vector           FFFE            Segment part 15 (?cstart)

    -------------------------------------------------------------------------
  LIBRARY MODULE, NAME : ?div64i

  SEGMENTS IN THE MODULE
  ======================
<CODE> 1 (was CODE)
  Relative segment, address: 756C - 7603 (0x98 bytes), align: 1
  Segment part 7.
           ENTRY                   ADDRESS         REF BY
           =====                   =======         ======
           _Div64u                 756C            _LitobLargeNoMb (?xprintflarge_nomb)
               CSTACK = 00000000 ( 0000001E )
    -------------------------------------------------------------------------
<CODE> 1 (was CODE)
  Relative segment, address: 9120 - 9131 (0x12 bytes), align: 1
  Segment part 8.             Intra module refs:   _Div64u
    -------------------------------------------------------------------------
<CODE> 1 (was CODE)
  Relative segment, address: 7D3E - 7DBB (0x7e bytes), align: 1
  Segment part 6.
           ENTRY                   ADDRESS         REF BY
           =====                   =======         ======
           _Mod64u                 7D3E            _LitobLargeNoMb (?xprintflarge_nomb)
               CSTACK = 00000000 ( 00000016 )
    -------------------------------------------------------------------------
<CODE> 1 (was CODE)
  Relative segment, address: 9144 - 9155 (0x12 bytes), align: 1
  Segment part 11.            Intra module refs:   _Div64u
                                                   _Mod64u
    -------------------------------------------------------------------------
<CODE> 1 (was CODE)
  Relative segment, address: 9156 - 915D (0x8 bytes), align: 1
  Segment part 9.             Intra module refs:   _Div64u
    -------------------------------------------------------------------------
<CODE> 1 (was CODE)
  Relative segment, address: 915E - 9167 (0xa bytes), align: 1
  Segment part 10.            Intra module refs:   Segment part 9
                                                   _Mod64u

    -------------------------------------------------------------------------
  LIBRARY MODULE, NAME : ?div

  SEGMENTS IN THE MODULE
  ======================
<CODE> 1 (was CODE)
  Relative segment, address: 9016 - 902B (0x16 bytes), align: 1
  Segment part 0.
           ENTRY                   ADDRESS         REF BY
           =====                   =======         ======
           div                     9016            _GenldLargeNoMb (?xprintflarge_nomb)

    -------------------------------------------------------------------------
  LIBRARY MODULE, NAME : ?exit

  SEGMENTS IN THE MODULE
  ======================
<CODE> 1 (was CODE)
  Relative segment, address: 9316 - 9319 (0x4 bytes), align: 1
  Segment part 2.
           ENTRY                   ADDRESS         REF BY
           =====                   =======         ======
           exit                    9316            Segment part 26 (?cstart)
               calls direct
               CSTACK = 00000000 ( 00000004 )

    -------------------------------------------------------------------------
  LIBRARY MODULE, NAME : ?Mul32fHw

  SEGMENTS IN THE MODULE
  ======================
<CODE> 1 (was CODE)
  Relative segment, address: 69B2 - 6AE7 (0x136 bytes), align: 1
  Segment part 0.
           ENTRY                   ADDRESS         REF BY
           =====                   =======         ======
           ?Mul32fHw               69B2            TDC720x_start2stopn (tdc720x_calculation)
                                                   _LdtobLargeNoMb (?xprintflarge_nomb)
                                                   handleHostCommand (host_interface)
                                                   scale (?xprintflarge_nomb)

    -------------------------------------------------------------------------
  LIBRARY MODULE, NAME : ?Cast32f32i

  SEGMENTS IN THE MODULE
  ======================
<CODE> 1 (was CODE)
  Relative segment, address: 7856 - 78E7 (0x92 bytes), align: 1
  Segment part 0.
           ENTRY                   ADDRESS         REF BY
           =====                   =======         ======
           _Cast32sto32f           7856            TDC720x_normlsb (tdc720x_calculation)
                                                   TDC720x_start2stopn (tdc720x_calculation)
           _Cast32uto32f           786A            _LdtobLargeNoMb (?xprintflarge_nomb)
                                                   handleHostCommand (host_interface)

    -------------------------------------------------------------------------
  LIBRARY MODULE, NAME : _Cast32fto32u

  SEGMENTS IN THE MODULE
  ======================
<CODE> 1 (was CODE)
  Relative segment, address: 9274 - 927F (0xc bytes), align: 1
  Segment part 0.
           ENTRY                   ADDRESS         REF BY
           =====                   =======         ======
           _Cast32fto32u           9274            _LdtobLargeNoMb (?xprintflarge_nomb)
                                                   handleHostCommand (host_interface)

    -------------------------------------------------------------------------
  LIBRARY MODULE, NAME : ?FLT_Extract

  SEGMENTS IN THE MODULE
  ======================
<CODE> 1 (was CODE)
  Relative segment, address: 872C - 8777 (0x4c bytes), align: 1
  Segment part 0.
           ENTRY                   ADDRESS         REF BY
           =====                   =======         ======
           ?FLT_Extract            872C            _Cast32fto32u (_Cast32fto32u)

    -------------------------------------------------------------------------
  LIBRARY MODULE, NAME : ?FLT_LT

  SEGMENTS IN THE MODULE
  ======================
<CODE> 1 (was CODE)
  Relative segment, address: 85EE - 863F (0x52 bytes), align: 1
  Segment part 0.
           ENTRY                   ADDRESS         REF BY
           =====                   =======         ======
           ?FLT_LT                 85EE            _CmpLt32f (_CmpLt32f)

    -------------------------------------------------------------------------
  LIBRARY MODULE, NAME : _CmpLt32f

  SEGMENTS IN THE MODULE
  ======================
<CODE> 1 (was CODE)
  Relative segment, address: 9296 - 929F (0xa bytes), align: 1
  Segment part 0.
           ENTRY                   ADDRESS         REF BY
           =====                   =======         ======
           _CmpLt32f               9296            _LdtobLargeNoMb (?xprintflarge_nomb)

    -------------------------------------------------------------------------
  LIBRARY MODULE, NAME : _Div32f

  SEGMENTS IN THE MODULE
  ======================
<CODE> 1 (was CODE)
  Relative segment, address: 6AE8 - 6C17 (0x130 bytes), align: 1
  Segment part 0.
           ENTRY                   ADDRESS         REF BY
           =====                   =======         ======
           _Div32f                 6AE8            TDC720x_normlsb (tdc720x_calculation)
                                                   _LdtobLargeNoMb (?xprintflarge_nomb)
                                                   handleHostCommand (host_interface)

    -------------------------------------------------------------------------
  LIBRARY MODULE, NAME : _Add32f

  SEGMENTS IN THE MODULE
  ======================
<CODE> 1 (was CODE)
  Relative segment, address: 6714 - 6875 (0x162 bytes), align: 1
  Segment part 0.
           ENTRY                   ADDRESS         REF BY
           =====                   =======         ======
           _Add32f                 6718            TDC720x_start2stopn (tdc720x_calculation)
                                                   handleHostCommand (host_interface)
           _Sub32f                 6714            _LdtobLargeNoMb (?xprintflarge_nomb)
                                                   handleHostCommand (host_interface)

    -------------------------------------------------------------------------
  LIBRARY MODULE, NAME : ?DivMod816u

  SEGMENTS IN THE MODULE
  ======================
<CODE> 1 (was CODE)
  Relative segment, address: 8EFA - 8F15 (0x1c bytes), align: 1
  Segment part 0.
           ENTRY                   ADDRESS         REF BY
           =====                   =======         ======
           ?DivMod8u               8EFA 
           ?DivMod16u              8EFE            Segment part 0 (?DivMod816s)
                                                   USB_determineFreq (usb)

    -------------------------------------------------------------------------
  LIBRARY MODULE, NAME : ?DivMod816s

  SEGMENTS IN THE MODULE
  ======================
<CODE> 1 (was CODE)
  Relative segment, address: 8B28 - 8B5B (0x34 bytes), align: 1
  Segment part 0.
           ENTRY                   ADDRESS         REF BY
           =====                   =======         ======
           ?DivMod8s               8B28 
           ?DivMod16s              8B2C            div (?div)
                                                   timer2_A0_init (timer_queue)

    -------------------------------------------------------------------------
  LIBRARY MODULE, NAME : ?DivMod32u

  SEGMENTS IN THE MODULE
  ======================
<CODE> 1 (was CODE)
  Relative segment, address: 8A84 - 8ABB (0x38 bytes), align: 1
  Segment part 0.
           ENTRY                   ADDRESS         REF BY
           =====                   =======         ======
           ?DivMod32u              8A84            ?DivMod32s (?DivMod32s)
                                                   Segment part 14 (?xprintflarge_nomb)

    -------------------------------------------------------------------------
  LIBRARY MODULE, NAME : ?DivMod32s

  SEGMENTS IN THE MODULE
  ======================
<CODE> 1 (was CODE)
  Relative segment, address: 8956 - 8995 (0x40 bytes), align: 1
  Segment part 0.
           ENTRY                   ADDRESS         REF BY
           =====                   =======         ======
           ?DivMod32s              8956            _LdtobLargeNoMb (?xprintflarge_nomb)

    -------------------------------------------------------------------------
  LIBRARY MODULE, NAME : ?memchr

  SEGMENTS IN THE MODULE
  ======================
<CODE> 1 (was CODE)
  Relative segment, address: 9000 - 9015 (0x16 bytes), align: 1
  Segment part 2.
           ENTRY                   ADDRESS         REF BY
           =====                   =======         ======
           __iar_Memchr            9000            _PrintfLargeNoMb (?xprintflarge_nomb)
               CSTACK = 00000000 ( 00000004 )

    -------------------------------------------------------------------------
  LIBRARY MODULE, NAME : ?memcpy

  SEGMENTS IN THE MODULE
  ======================
<CODE> 1 (was CODE)
  Relative segment, address: 90D8 - 90E9 (0x12 bytes), align: 1
  Segment part 2.
           ENTRY                   ADDRESS         REF BY
           =====                   =======         ======
           memcpy                  90D8            Segment part 11 (?xprintflarge_nomb)
                                                   _GenldLargeNoMb (?xprintflarge_nomb)
                                                   _LdtobLargeNoMb (?xprintflarge_nomb)
                                                   __data16_memcpy (?memzero)
               CSTACK = 00000000 ( 00000004 )

    -------------------------------------------------------------------------
  LIBRARY MODULE, NAME : ?ClearMemoryWords

  SEGMENTS IN THE MODULE
  ======================
<CODE> 1 (was CODE)
  Relative segment, address: 91A8 - 91B7 (0x10 bytes), align: 1
  Segment part 0.
           ENTRY                   ADDRESS         REF BY
           =====                   =======         ======
           ?ClearMemoryWords       91A8            USB_initMemcpy (usbdma)

    -------------------------------------------------------------------------
  LIBRARY MODULE, NAME : ?memset

  SEGMENTS IN THE MODULE
  ======================
<CODE> 1 (was CODE)
  Relative segment, address: 9090 - 90A1 (0x12 bytes), align: 1
  Segment part 2.
           ENTRY                   ADDRESS         REF BY
           =====                   =======         ======
           memset                  9090            CdcResetData (UsbCdc)
               CSTACK = 00000000 ( 00000004 )

    -------------------------------------------------------------------------
  LIBRARY MODULE, NAME : ?memzero

  SEGMENTS IN THE MODULE
  ======================
<CODE> 1 (was CODE)
  Relative segment, address: 90A2 - 90B3 (0x12 bytes), align: 1
  Segment part 4.
           ENTRY                   ADDRESS         REF BY
           =====                   =======         ======
           __data16_memzero        90A2            ?cstart_init_zero (?cstart)
               CSTACK = 00000000 ( 00000004 )
    -------------------------------------------------------------------------
<CODE> 1 (was CODE)
  Relative segment, address: 9322 - 9325 (0x4 bytes), align: 1
  Segment part 3.
           ENTRY                   ADDRESS         REF BY
           =====                   =======         ======
           __data16_memcpy         9322            ?cstart_init_copy (?cstart)
               calls direct
               CSTACK = 00000000 ( 00000004 )

    -------------------------------------------------------------------------
  LIBRARY MODULE, NAME : ?Mul32Hw32

  SEGMENTS IN THE MODULE
  ======================
<CODE> 1 (was CODE)
  Relative segment, address: 8DF6 - 8E19 (0x24 bytes), align: 1
  Segment part 0.
           ENTRY                   ADDRESS         REF BY
           =====                   =======         ======
           ?Mul32Hw32              8DF6            _LdtobLargeNoMb (?xprintflarge_nomb)

    -------------------------------------------------------------------------
  LIBRARY MODULE, NAME : ?IndCallR11

  SEGMENTS IN THE MODULE
  ======================
<CODE> 1 (was CODE)
  Relative segment, address: 92FE - 9301 (0x4 bytes), align: 1
  Segment part 0.
           ENTRY                   ADDRESS         REF BY
           =====                   =======         ======
           ?IndCallR11             92FE            _PutcharLargeNoMb (?xprintflarge_nomb)

    -------------------------------------------------------------------------
  LIBRARY MODULE, NAME : ?IndCallR15

  SEGMENTS IN THE MODULE
  ======================
<CODE> 1 (was CODE)
  Relative segment, address: 932A - 932D (0x4 bytes), align: 1
  Segment part 0.
           ENTRY                   ADDRESS         REF BY
           =====                   =======         ======
           ?IndCallR15             932A            USB_init (usb)
                                                   usbDecodeAndProcessUsbRequest (usb)

    -------------------------------------------------------------------------
  LIBRARY MODULE, NAME : ?sprintf

  SEGMENTS IN THE MODULE
  ======================
<CODE> 1 (was CODE)
  Relative segment, address: 8850 - 8891 (0x42 bytes), align: 1
  Segment part 2.
           ENTRY                   ADDRESS         REF BY
           =====                   =======         ======
           sprintf                 8850            handleHostCommand (host_interface)
                                                   print_start2stopn (tdc720x_calculation)
               calls direct
               CSTACK = 00000000 ( 0000000C )

    -------------------------------------------------------------------------
  LIBRARY MODULE, NAME : ?strchr

  SEGMENTS IN THE MODULE
  ======================
<CODE> 1 (was CODE)
  Relative segment, address: 9198 - 91A7 (0x10 bytes), align: 1
  Segment part 2.
           ENTRY                   ADDRESS         REF BY
           =====                   =======         ======
           __iar_Strchr            9198            _PrintfLargeNoMb (?xprintflarge_nomb)
               CSTACK = 00000000 ( 00000004 )

    -------------------------------------------------------------------------
  LIBRARY MODULE, NAME : ?strlen

  SEGMENTS IN THE MODULE
  ======================
<CODE> 1 (was CODE)
  Relative segment, address: 90C6 - 90D7 (0x12 bytes), align: 1
  Segment part 2.
           ENTRY                   ADDRESS         REF BY
           =====                   =======         ======
           strlen                  90C6            _PrintfLargeNoMb (?xprintflarge_nomb)
                                                   handleHostCommand (host_interface)
                                                   print_start2stopn (tdc720x_calculation)
               CSTACK = 00000000 ( 00000004 )

    -------------------------------------------------------------------------
  LIBRARY MODULE, NAME : ?xdunscal

  SEGMENTS IN THE MODULE
  ======================
<CODE> 1 (was CODE)
  Relative segment, address: 8778 - 87C1 (0x4a bytes), align: 1
  Segment part 2.
           ENTRY                   ADDRESS         REF BY
           =====                   =======         ======
           __iar_Dunscale          8778            _LdtobLargeNoMb (?xprintflarge_nomb)
               CSTACK = 00000000 ( 00000004 )

    -------------------------------------------------------------------------
  LIBRARY MODULE, NAME : ?xprintflarge_nomb

  SEGMENTS IN THE MODULE
  ======================
<CODE> 1 (was CODE)
  Relative segment, address: 5204 - 5713 (0x510 bytes), align: 1
  Segment part 25.
           ENTRY                   ADDRESS         REF BY
           =====                   =======         ======
           _PrintfLargeNoMb        5204            sprintf (?sprintf)
               calls direct
               CSTACK = 00000000 ( 00000074 )
    -------------------------------------------------------------------------
<CODE> 1 (was CODE)
  Relative segment, address: 91E4 - 91F1 (0xe bytes), align: 1
  Segment part 29.            Intra module refs:   _PrintfLargeNoMb
    -------------------------------------------------------------------------
<CODE> 1 (was CODE)
  Relative segment, address: 925C - 9267 (0xc bytes), align: 1
  Segment part 30.            Intra module refs:   _PrintfLargeNoMb
    -------------------------------------------------------------------------
<CODE> 1 (was CODE)
  Relative segment, address: 92AA - 92B3 (0xa bytes), align: 1
  Segment part 31.            Intra module refs:   _PrintfLargeNoMb
    -------------------------------------------------------------------------
<CODE> 1 (was CODE)
  Relative segment, address: 9200 - 9201 (0x2 bytes), align: 1
  Segment part 32.            Intra module refs:   _PrintfLargeNoMb
    -------------------------------------------------------------------------
<CODE> 1 (was CODE)
  Relative segment, address: 9202 - 920D (0xc bytes), align: 1
  Segment part 33.            Intra module refs:   Segment part 32
                                                   _PrintfLargeNoMb
    -------------------------------------------------------------------------
<CODE> 1 (was CODE)
  Relative segment, address: 7C3E - 7CB5 (0x78 bytes), align: 1
  Segment part 21.            Intra module refs:   _PrintfLargeNoMb
           LOCAL                   ADDRESS         
           =====                   =======         
           LoadInt                 7C3E 
               CSTACK = 00000000 ( 00000004 )
    -------------------------------------------------------------------------
<CODE> 1 (was CODE)
  Relative segment, address: 7CB6 - 7CBF (0xa bytes), align: 1
  Segment part 22.            Intra module refs:   LoadInt
                                                   _LitobLargeNoMb
                                                   _PrintfLargeNoMb
    -------------------------------------------------------------------------
<CODE> 1 (was CODE)
  Relative segment, address: 928C - 9295 (0xa bytes), align: 1
  Segment part 23.            Intra module refs:   LoadInt
                                                   _LdtobLargeNoMb
                                                   _PrintfLargeNoMb
    -------------------------------------------------------------------------
<CODE> 1 (was CODE)
  Relative segment, address: 9244 - 924F (0xc bytes), align: 1
  Segment part 24.            Intra module refs:   LoadInt
    -------------------------------------------------------------------------
<CODE> 1 (was CODE)
  Relative segment, address: 8ABC - 8AF1 (0x36 bytes), align: 1
  Segment part 20.            Intra module refs:   Segment part 33
           LOCAL                   ADDRESS         
           =====                   =======         
           pad                     8ABC 
               calls direct
               CSTACK = 00000000 ( 00000012 )
    -------------------------------------------------------------------------
<CODE> 1 (was CODE)
  Relative segment, address: 6102 - 62B5 (0x1b4 bytes), align: 1
  Segment part 16.            Intra module refs:   _PrintfLargeNoMb
           LOCAL                   ADDRESS         
           =====                   =======         
           _LitobLargeNoMb         6102 
               calls direct
               CSTACK = 00000000 ( 0000002A )
    -------------------------------------------------------------------------
<CODE> 1 (was CODE)
  Relative segment, address: 920E - 921B (0xe bytes), align: 1
  Segment part 17.            Intra module refs:   _LitobLargeNoMb
    -------------------------------------------------------------------------
<CODE> 1 (was CODE)
  Relative segment, address: 9132 - 9143 (0x12 bytes), align: 1
  Segment part 18.            Intra module refs:   _LitobLargeNoMb
    -------------------------------------------------------------------------
<CODE> 1 (was CODE)
  Relative segment, address: 907C - 908F (0x14 bytes), align: 1
  Segment part 19.            Intra module refs:   _LitobLargeNoMb
    -------------------------------------------------------------------------
<CODE> 1 (was CODE)
  Relative segment, address: 88D4 - 8915 (0x42 bytes), align: 1
  Segment part 15.            Intra module refs:   _LdtobLargeNoMb
           LOCAL                   ADDRESS         
           =====                   =======         
           scale                   88D4 
               calls direct
               CSTACK = 00000000 ( 00000010 )
    -------------------------------------------------------------------------
<CODE> 1 (was CODE)
  Relative segment, address: 5C48 - 5EA5 (0x25e bytes), align: 1
  Segment part 13.            Intra module refs:   _PrintfLargeNoMb
           LOCAL                   ADDRESS         
           =====                   =======         
           _LdtobLargeNoMb         5C48 
               calls direct
               CSTACK = 00000000 ( 0000004A )
    -------------------------------------------------------------------------
<CODE> 1 (was CODE)
  Relative segment, address: 90EA - 90FB (0x12 bytes), align: 1
  Segment part 14.            Intra module refs:   _LdtobLargeNoMb
    -------------------------------------------------------------------------
<CODE> 1 (was CODE)
  Relative segment, address: 59D8 - 5C47 (0x270 bytes), align: 1
  Segment part 10.            Intra module refs:   _LdtobLargeNoMb
           LOCAL                   ADDRESS         
           =====                   =======         
           _GenldLargeNoMb         59D8 
               calls direct
               CSTACK = 00000000 ( 00000020 )
    -------------------------------------------------------------------------
<CODE> 1 (was CODE)
  Relative segment, address: 9178 - 9187 (0x10 bytes), align: 1
  Segment part 11.            Intra module refs:   _GenldLargeNoMb
    -------------------------------------------------------------------------
<CODE> 1 (was CODE)
  Relative segment, address: 9168 - 9177 (0x10 bytes), align: 1
  Segment part 12.            Intra module refs:   _GenldLargeNoMb
    -------------------------------------------------------------------------
<CODE> 1 (was CODE)
  Relative segment, address: 8DCE - 8DF5 (0x28 bytes), align: 1
  Segment part 9.             Intra module refs:   _PrintfLargeNoMb
                                                   _PutcharsLargeNoMb
           LOCAL                   ADDRESS         
           =====                   =======         
           _PutcharLargeNoMb       8DCE 
               calls indirect
               CSTACK = 00000000 ( 0000000C )
    -------------------------------------------------------------------------
<CODE> 1 (was CODE)
  Relative segment, address: 8D24 - 8D4F (0x2c bytes), align: 1
  Segment part 8.             Intra module refs:   Segment part 30
                                                   pad
           LOCAL                   ADDRESS         
           =====                   =======         
           _PutcharsLargeNoMb      8D24 
               calls direct
               CSTACK = 00000000 ( 00000010 )
    -------------------------------------------------------------------------
<CODE> 1 (was CODE)
  Relative segment, address: 91B8 - 91C7 (0x10 bytes), align: 1
  Segment part 26.            Intra module refs:   _PrintfLargeNoMb
    -------------------------------------------------------------------------
<CODE> 1 (was CODE)
  Relative segment, address: 90FC - 910D (0x12 bytes), align: 1
  Segment part 27.            Intra module refs:   _PrintfLargeNoMb
    -------------------------------------------------------------------------
<CODE> 1 (was CODE)
  Relative segment, address: 91D6 - 91E3 (0xe bytes), align: 1
  Segment part 28.            Intra module refs:   _PrintfLargeNoMb
    -------------------------------------------------------------------------
DATA16_C
  Relative segment, address: 4668 - 466E (0x7 bytes), align: 0
  Segment part 2.             Intra module refs:   _PrintfLargeNoMb
    -------------------------------------------------------------------------
DATA16_C
  Relative segment, address: 466F - 4672 (0x4 bytes), align: 0
  Segment part 3.             Intra module refs:   _LdtobLargeNoMb
    -------------------------------------------------------------------------
DATA16_C
  Relative segment, address: 4673 - 4676 (0x4 bytes), align: 0
  Segment part 4.             Intra module refs:   _LdtobLargeNoMb
    -------------------------------------------------------------------------
DATA16_C
  Relative segment, address: 4677 - 467A (0x4 bytes), align: 0
  Segment part 5.             Intra module refs:   _LdtobLargeNoMb
    -------------------------------------------------------------------------
DATA16_C
  Relative segment, address: 467B - 467E (0x4 bytes), align: 0
  Segment part 6.             Intra module refs:   _LdtobLargeNoMb
    -------------------------------------------------------------------------
DATA16_C
  Relative segment, address: 467F - 4680 (0x2 bytes), align: 0
  Segment part 7.             Intra module refs:   _GenldLargeNoMb

    -------------------------------------------------------------------------
  LIBRARY MODULE, NAME : ?xsprout

  SEGMENTS IN THE MODULE
  ======================
<CODE> 1 (was CODE)
  Relative segment, address: 9188 - 9197 (0x10 bytes), align: 1
  Segment part 2.
           ENTRY                   ADDRESS         REF BY
           =====                   =======         ======
           _SProut                 9188            sprintf (?sprintf)
               CSTACK = 00000000 ( 00000004 )




                ****************************************
                *                                      *
                *            MODULE SUMMARY            *
                *                                      *
                ****************************************

Module                         CODE      DATA      CONST
------                         ----      ----      -----
                              (Rel)  (Rel)  (Abs)  (Rel)
?Cast32f32i                     146
?ClearMemoryWords                16
?DivMod32s                       64
?DivMod32u                       56
?DivMod816s                      52
?DivMod816u                      28
?FLT_Extract                     76
?FLT_LT                          82
?IndCallR11                       4
?IndCallR15                       4
?Mul32Hw32                       36
?Mul32fHw                       310
?__dbg_break                      2
?__exit                          22
?_exit                            4
?cstart                          40
?div                             22
?div64i                         332
?exit                             4
?memchr                          22
?memcpy                          18
?memset                          18
?memzero                         22
?reset_vector                     2
?sprintf                         66
?strchr                          16
?strlen                          18
?xdunscal                        74
?xprintflarge_nomb            3 518                   25
?xsprout                         16
HAL_FLASH                                       4
HAL_PMAP                                        4
HAL_PMM                         454            10
HAL_UCS
  + shared                                     14
TI_MSP430_spi_USCIB0_5xx        952             9
  + shared                                      2
UsbCdc                        2 780     34      1
UsbIsr                          696             2
  + common                      104
_Add32f                         354
_Cast32fto32u                    12
_CmpLt32f                        10
_Div32f                         304
descriptors                                          509
dma                             298
gpio                             42                   28
host_interface                2 522     47      2     15
  + shared                                     18
main                          1 008    211     18      5
  + shared                      124             6
  + common
tdc720x_calculation             500    212            37
tdc720x_measurement_control     318      1
tdc720x_mode1_lt12ns            402
timer_queue                     268      8     30      2
  + common                      108
tlv                              80
uart_commn                      106            10
ucs                              74
usb                           2 864     69    152     33
  + shared                                     10
usbConstructs                   188
usbEventHandling                 72
usbdma                          234      8
N/A (command line)                     240
N/A (alignment)
----------                   ------    ---    ---    ---
Total:                       19 628    830    292    654
  + common                      124


                ****************************************
                *                                      *
                *      SEGMENTS IN ADDRESS ORDER       *
                *                                      *
                ****************************************


SEGMENT              SPACE    START ADDRESS   END ADDRESS     SIZE  TYPE  ALIGN
=======              =====    =============   ===========     ====  ====  =====
DATA16_AN                              0102 - 0103               2   rel    0
                                       0120 - 0121               2 
                                       0124 - 0127               4 
                                       012C - 012F               4 
                                       0140 - 0141               2 
                                       0144 - 0145               2 
                                       015C - 015D               2 
                                       0160 - 016F              10 
                                       0198 - 019B               4 
                                       01C0 - 01C3               4 
                                       0200 - 020B               C 
                                       0218 - 0219               2 
                                       021C - 021D               2 
                                       0222 - 0227               6 
                                       022A - 022B               2 
                                       0242 - 0245               4 
                                       024A - 024B               2 
                                       0262 - 0265               4 
                                       0340 - 0343               4 
                                       0352 - 0353               2 
                                       0380 - 0383               4 
                                       0392 - 0393               2 
                                       03A0 - 03A1               2 
                                       0400 - 0407               8 
                                       0412 - 0417               6 
                                       05E0 - 05E1               2 
                                       05E6 - 05E7               2 
                                       05EA - 05EA               1 
                                       05EC - 05EC               1 
                                       05EE - 05EE               1 
                                       05FC - 05FD               2 
                                       0600 - 0601               2 
                                       0606 - 0608               3 
                                       060E - 060E               1 
                                       061C - 061D               2 
                                       0620 - 0621               2 
                                       0626 - 0627               2 
                                       062A - 062A               1 
                                       062C - 062C               1 
                                       063C - 063D               2 
                                       0900 - 0905               6 
                                       0908 - 0909               2 
                                       0910 - 0915               6 
                                       0920 - 0923               4 
                                       092E - 0930               3 
                                       0932 - 0933               2 
                                       093C - 093F               4 
                                       2370 - 23BF              50 
                                       23C8 - 23FF              38 
DATA16_I                               2400 - 240C               D   rel    1
DATA16_Z                               240E - 262C             21F   rel    1
DATA16_N                               262D - 264E              22   rel    0
DATA20_Z                                  2650                       rel    1
DATA20_I                                  2650                       rel    1
CODE_I                                    2650                       rel    1
DATA20_N                                  2650                       rel    1
DATA20_HEAP                            2650 - 269F              50   rel    1
CSTACK                                 4360 - 43FF              A0   rel    1
DATA16_C                               4400 - 4680             281   rel    1
DATA16_ID                              4682 - 468E               D   rel    1
CSTART                                 4690 - 46B7              28   rel    1
ISR_CODE                               46B8 - 4861             1AA   rel    1
<CODE> 1                               4862 - 9339            4AD8   rel    1
CODE_ID                                   933A                       rel    1
DATA20_C                                  933A                       rel    1
DATA20_ID                                 933A                       rel    1
INTVEC                                 FF80 - FFFB              7C   com    1
RESET                                  FFFE - FFFF               2   rel    1

                ****************************************
                *                                      *
                *        END OF CROSS REFERENCE        *
                *                                      *
                ****************************************

 19 752 bytes of CODE  memory
    830 bytes of DATA  memory (+ 292 absolute )
    654 bytes of CONST memory

Errors: none
Warnings: none

